:1080000000000120C10C01003DE400003DE400003F
:108010003DE400003DE400003DE4000000000000FD
:108020000000000000000000000000003DE400002F
:108030003DE40000000000003DE400001D8600005B
:108040003DE400003DE400003DE400003DE40000AC
:108050003DE400003DE400003DE400003DE400009C
:108060003DE400003DE400003DE400003DE400008C
:108070003DE400003DE400003DE400003DE400007C
:108080003DE400003DE400003DE400003DE400006C
:108090003DE400003DE400003DE400003DE400005C
:1080A0003DE4000051D300003DE400003DE4000049
:1080B0003DE400003DE400003DE400003DE400003C
:1080C0003DE400003DE400003DE400003DE400002C
:1080D0003DE400003DE400003DE4000065CF000009
:1080E0003DE400003DE400003DE400003DE400000C
:1080F0003DE400003DE400003DE400003DE40000FC
:108100003DE400003DE400003DE400003DE40000EB
:108110003DE4000059F600003DE400003DE40000AD
:108120003DE400003DE400003DE400003DE40000CB
:108130003DE400003DE400003DE400003DE40000BB
:108140003DE400003DE40000718700003DE40000D4
:108150003DE400003DE400003DE400003DE400009B
:108160003DE40000A1CF00003DE400003DE400003C
:108170003DE400003DE400003DE400003DE400007B
:088180003DE400003DE40000B5
:10840000FFFFFFFFFFFFFFFFFFFFFFFF7EF9FFFF03
:1084100010B5054C237833B9044B13B10448AFF3BE
:1084200000800123237010BD0086FF1F00000000A4
:10843000A41401000C4B43B10C480D4910B5AFF327
:1084400000800C48036823B910BD0A48036833B99B
:108450007047094B002BF7D0BDE810401847064B7A
:10846000002BF5D0184700BF00000000A414010045
:108470000486FF1F6C85FF1F0000000080F3118839
:1084800070472F4B41F238015A5842F478525A50F3
:108490002C4A927902F00C020C2A4FD041F244028D
:1084A0002949995003F558339A78110748BF9A78AB
:1084B000264944BF42F008029A70214B41F244021F
:1084C000995041F204015A5842F4803242F0C002FD
:1084D0005A501A6842F440221A6003F5E833242205
:1084E0005A701B4A80211170A2221A70DA7802F0A9
:1084F0001F02DA7003221A7100225A719A799207C8
:10850000FCD59A79D006FCD40E4B19469A7902F024
:108510000C02082AFAD140225A718B7903F00C031D
:10852000082BFAD1074B1A4699794906FCD5222126
:108530001970937903F00C030C2BFAD1704700BF2C
:1085400000700440004006400000330100001301A9
:10855000005006402B4B5A7902F0E0025A711A790A
:1085600002F0F8021A71284A136843F004031360FA
:10857000264A136823F0784323F001031360244B49
:108580001A7802F08C0242F050021A705A7802F007
:108590009C0242F040025A709A7802F0E6029A7009
:1085A0001C4A0023137083F311881B4B012283F8AC
:1085B000182383F81923022283F83C2383F83D23F0
:1085C00083F84B2383F84C2383F84D2383F84E2301
:1085D00083F84F23032283F81F2383F8212383F892
:1085E000232383F8252383F84223042283F82723B7
:1085F000052283F84923062283F83B23072283F8C8
:108600003523704700F007404080044000D0004010
:1086100000D0074000E0074000E100E00C4A13688A
:10862000013313600B4A1368013313600A4B1A6855
:108630003AB11A68013A1A601B6813B9074B012254
:108640001A70074B1A6812B11A68013A1A6070471B
:108650001C86FF1F6C98FF1FB493FF1FB093FF1F72
:10866000B893FF1F024B034A5A6007221A607047F3
:1086700010E000E000770100014B1868704700BF70
:108680001C86FF1F1449154B41F22802072888BF9A
:10869000002010B553F82030114CB4FBF3F48B5884
:1086A00043F480638B500F4B4FF440729A63422027
:1086B000DA6305F0E1FE0C4B0022DA709A709A71D1
:1086C000DA725A71C4F30422E4B21A705C70DA7878
:1086D00042F02C02DA7010BD0070044068120100F4
:1086E000C0C62D0000B0044000A00E40094A136827
:1086F00051680133202B08BF00238B4208D011683A
:10870000114408721360044AD37843F08003D37095
:10871000704700BF2086FF1F00A00E400A4B996AD9
:10872000DA6A91420DD09A6A511C1A44996292F801
:10873000302002709A6A202A01D100229A62012018
:1087400070470020704700BF2086FF1F044B1A7837
:1087500002F0FF0012B100221A700120704700BF22
:10876000B093FF1F014B1865704700BF2086FF1FA5
:1087700030B526480179C9B28C0617D5244BDA6A80
:108780009C6A0132202A08BF0022A2421BBFDC6A79
:10879000C579C27918191EBFEDB280F83050DA627F
:1087A0001C4A052010601A6D1B4B1A604A0608D53A
:1087B0001A4B4FF480529A60144AD37803F0BF03E7
:1087C000D3700B061BD5144B1868C0B9104B196831
:1087D0005A68914214D0114A4FF4805151605A683E
:1087E000511C1A445960117A084AC9B2D1715968AA
:1087F000202908BF5860D37843F04003D37030BDC0
:10880000024AD37803F07F03F8E700BF00A00E40D0
:108810002086FF1FB493FF1FB893FF1F80F00F4007
:1088200062B67047FFF7FCBF72B67047FFF7FCBF38
:108830004FF0E02318B1034AC3F80C2D7047024AE9
:10884000FAE700BF0400FA050100FA05F7B543484E
:10885000434C444D444E4FF480730E22436083607A
:10886000A2606261414A53629364D36413655365A5
:1088700093654FF4F0026A61AA603D4A4FF490712B
:1088800051621363936402F5342280324FF49051A5
:1088900091604FF48021516001F590515161354A4A
:1088A00040F20311116051609160D160116151611A
:1088B0009161D161304900224A6130490B614B61BD
:1088C0008B618B6601F5322101F580718E604E61FE
:1088D00003600826C360134611460A202A46B446A0
:1088E0001F46A646C4F804C00197019DB5F57A7FDE
:1088F0002AD3DEF81050A660ED0748BF013101977A
:10890000019DB5F57A7F23D3DEF81050ED0758BFEF
:1089100001330138E6D10A2919491DD10A2B1BD18F
:1089200001230B700D4B4FF4E0611960D96003F522
:1089300080534FF48071196001235360536943F0F1
:108940000103536103B0F0BD019D01350195CCE7F2
:10895000019D01350195D3E70023E2E70090044033
:1089600000F00F4040F00F407000000400A00440F1
:1089700000B0044000C00440C0F00F4000D00440EC
:10898000F293FF1FF7B5104B1B78D3B10F4B104D6F
:1089900002210F46042000241E469F605860019467
:1089A000019AAA4209D97160B0600194019AAA4261
:1089B000F3D8019A01320192F8E7019A013201924B
:1089C000EEE703B0F0BD00BFF293FF1F00F00F40D1
:1089D0001FA10700032806D8DFE800F00206080AF6
:1089E0001022054B5A6070472022FAE74022F8E730
:1089F0004FF08062F5E700BF00F10F40032806D872
:108A0000DFE800F00206080A1022054B9A60704762
:108A10002022FAE74022F8E74FF08062F5E700BF36
:108A200000F10F4010B50021044644FA01F3DB07C2
:108A3000C8B205D5FFF7CEFF01310829F5D110BD29
:108A4000FFF7DCFFF8E708B5032813D8DFE800F0EC
:108A5000020C0E10002004F009FB43F27C03984244
:108A600094BF0020012008BD0120F4E70220F2E7B6
:108A70000320F0E7002008BD032817D8DFE800F046
:108A800002070C110A4B1868C0F300107047084B1E
:108A90001868C0F340107047054B1868C0F3801089
:108AA0007047034B1868C0F3806070470020704720
:108AB00000F10F4070B5002425460126E0B2FFF713
:108AC000C2FF18B106FA04F31D43EDB20134082CBD
:108AD000F4D1284670BD024B1869C043C0B270473C
:108AE000C0F00F4008B5082004F0C0FA5E280ED987
:108AF000104B1A780AB901221A70082004F0B6FA4D
:108B000063280CD90C4B4FF400725A6008BD082042
:108B100004F0ACFA5428F0D80022064BECE7082009
:108B200004F0A4FA54289EBF034B4FF400729A60DD
:108B300008BD00BF7486FF1F80F00F40034B1878FC
:108B4000013801288CBF0020012070477486FF1F68
:108B5000034B1878012806BF02221A7000207047C4
:108B60007486FF1FC0B205F0BBBAC0B205F0A6BA4A
:108B70000B4B10F0010F4FF4800214BF5A609A6043
:108B800010F0020F4FF4001214BF5A609A6010F0F8
:108B9000040F4FF4801214BF5A609A60704700BFF0
:108BA00040F00F4008B507F07BFB05F039FE05F0FB
:108BB000E9FDBDE8084007F0F5BB38B5054605F00E
:108BC00037FD08280AD900242819013405F0B0FD22
:108BD000092CF9D105F0E0FD012038BD002038BD99
:108BE000092105F045BD002005F0D2BF22492348E8
:108BF00041F23C028B5843F440538B50204B0121EF
:108C000019601A6802431A601E4ADA601A61DA6A49
:108C100042F08052DA621A6822F001021A601A6881
:108C200022F000621A60184A4FF400731360536018
:108C30009360D360136153619361D361A2F5F03205
:108C400011601168014311601049D16001F52001E4
:108C50001161D16A41F08051D162116821F00101A6
:108C60001160116821F00061116002F5E832936231
:108C7000D36213645364704700700440000C1F807B
:108C800000C002400300013E00B004400400513E19
:108C9000FF2810B54FEA004323D82B4C03F47C1374
:108CA0008AB141F000610B436363E36A002BFCDA95
:108CB000254BDA6AD000FCD5986BDA6A42F0104294
:108CC000C0B2DA6210BD41F000410B436363E36A56
:108CD000002BFCDAA06BE36A43F01043C0B2E362FE
:108CE00010BDB0F5007F17D2184C03F47C135AB1B5
:108CF00041F000610B436363E36A002BFCDA134B22
:108D0000DA6AD100FCD5D7E741F000410B43636339
:108D1000E36A002BFCDADDE70D4C03F47C135AB157
:108D200041F000610B436363E36A002BFCDA084BFC
:108D3000DA6AD200FCD5BFE741F000410B43636320
:108D4000E36A002BFCDAC5E700C0024000D0024015
:108D500000C00A4010B5FFF78FFC0446FFF78CFCFB
:108D6000001B0028B8BF40420628F7DD10BD07B53C
:108D7000030A8DF805008DF80610032201A9A02032
:108D80008DF8043004F07AFBFFF7E4FF03B05DF8E0
:108D900004FBF0B5154600228BB00F461446AC42DA
:108DA00001D10BB0F0BD0AAB1344395D03F8221CAE
:108DB000531CC618F10602D0691E8C420DD1030A5D
:108DC0008DF80500033201A9A0208DF8043004F0CD
:108DD00055FBFFF7BFFF3046002301341A46DEE79C
:108DE0001FB5030A8DF80C30022203AB8DF80D007D
:108DF00000921946A02004F08DFB9DF80C0005B0F0
:108E00005DF804FB1FB5030A8DF80C308DF80D00DA
:108E100000920B46022203A9A02004F07BFB05B0C0
:108E20005DF804FBC0EBC000072200F5B040FFF77F
:108E3000B0BFC0EBC000072200F5B040FFF7E2BFB3
:108E400030B500238BB001AD1A465A550133222BA1
:108E5000FBD14FF4B044230A8DF805402222294665
:108E6000A02020348DF8043004F008FBFFF772FFD7
:108E7000B4F5803FEFD10BB030BD13B50C46C0EB5D
:108E8000C0000722694600F5B040FFF7BBFF9DF820
:108E9000002023789A4212D19DF8012063789A42EB
:108EA0000DD19DF80220A3789A4208D1DDF8030085
:108EB000D4F80330C31A5842584102B010BD002004
:108EC000FBE7704773B545F2FF70FFF789FF552840
:108ED00002D1284B1B78CBB3002145F2FF70FFF77E
:108EE00046FFFFF7ADFF40222349244D0020FFF746
:108EF00050FF40242046402229464034FFF749FFD6
:108F0000B4F5E07FF6D102AD002345F8043D4FF4FF
:108F1000D36440F678062046042229460434FFF73D
:108F200038FFB442F7D1002301934FF4FF6440F6B9
:108F3000D8062046042229460434FFF72AFFB4420B
:108F4000F7D1552145F2FF70FFF711FF40220A4982
:108F50000B4D0020FFF756FF4024A4F140012046AE
:108F6000402229444034FFF74DFFB4F5E07FF4D1AF
:108F700002B070BDF293FF1F0C80FF1F981201001A
:108F80000894FF1F044B9B78052B044B8CBF0422D5
:108F900003221A70704700BF5896FF1F7098FF1F7A
:108FA000F7B5CF4EB4787278052C354603D9042234
:108FB000CC4B1A7019E2A22A00F0458300F2F3802C
:108FC000132A00F08C8278D8072A00F0108238D853
:108FD000022A00F0B18107D8002A00F09781012A07
:108FE00000F0A3810322E3E7052A00F0C98100F223
:108FF000DE81042AF6D1D6F80300BB4E002856F8CD
:109000002430B8BF4042984706EB8404A061A8789A
:10901000202400F0010104FA01F1C9B2400804F073
:1090200049FB002840F0E181A87806EB800600F0BB
:10903000010104FA01F1B26941F00701C9B2400827
:109040006EE10F2A00F0258222D80D2A00F0EB8174
:1090500000F204820C2AC5D1202604F0010106FA90
:1090600001F141F01401C9B2600804F023FBAB78B0
:10907000D5F8032003F0010106FA01F141F01401D3
:10908000002A40F0CD8140F00202C9B2580847E101
:10909000112A04F001074FEA5406934800F01482A5
:1090A00040F2058200EB8404D5F80300236B984757
:1090B0002021B94041F00A0102E21A2A00F0608240
:1090C00030D8162A00F025820BD8142A00F014821A
:1090D000152A87D104F001032021994041F00C01A9
:1090E0001AE1182A04F001064FEA540700F02C8216
:1090F00040F21C82202404FA06F141F01401C9B2A6
:10910000384604F0D7FAAB78D5F8032003F0010114
:1091100004FA01F141F01401002A00F02E8240F01F
:109120000402B2E7202A00F0588222D81C2A00F05C
:109130004B82C0F040821F2A7FF454AF04F001013B
:10914000202606FA01F141F01001C9B2600804F0CE
:10915000B1FAAC78EB7804F00101C2B206FA01F181
:10916000C0F3072041F010010192009003F00F03BB
:1091700036E17F2A00F047828C2A00F05982212AAA
:109180007FF430AF210101F0100141F06E01600861
:1091900004F090FAB478C0B201902101F378009302
:1091A00001F010012AE2B52A00F0C58248D8A92AA8
:1091B00000F08B8220D8A52A00F057820ED8A32A6F
:1091C00000F04A82A42A7FF40DAFD6F8031020469F
:1091D000C9B203B0BDE8F04004F0D0BBA72A00F04C
:1091E0006B8240F25682D6F803102046C9B203B013
:1091F000BDE8F04004F05ABDAD2A00F081820DD8E0
:10920000AB2A00F0748240F26982D6F8031020463F
:10921000C9B203B0BDE8F04004F01BBDB12A00F0B4
:109220007882B32A00F07E82AE2A7FF4DBAED6F8D5
:1092300003102046C9B203B0BDE8F04004F020BDE1
:10924000C32A00F0B8822AD8BB2A00F0918215D830
:10925000B82A00F07B82B92A00F08182B62A7FF416
:10926000C1AE214BD6F8030053F82430984704F0E0
:1092700001032021994041F011017FE0C12A00F053
:10928000898200F28E82BC2A7FF4ACAED6F803103D
:109290002046C9B203B0BDE8F04004F0EDBDD12ACC
:1092A00000F0A08222D8CA2A00F09082CC2A00F0D6
:1092B0006882C92A7FF496AE1821600804F0FAF992
:1092C00000F48062B078D6F8033000F00104202169
:1092D00023F48063A14041F018011A43AEE600BFB9
:1092E0005896FF1F7098FF1F7886FF1FD42A00F042
:1092F0008182FF2A00F08582D22A7FF473AEC74BA9
:10930000D6F8032003EB8413DA6165E204F001036D
:109310002021994041F00D01D5F80320C9B2600821
:1093200003B0BDE8F04004F07DB904F00103202152
:10933000994041F00101EFE7D6F803302021002BDE
:1093400004F0010301FA03F14FEA5400C8BF0122FF
:10935000C9B204F067F9B478B14BD6F80300012222
:109360001A55B04B002853F82430B8BF40429847F4
:1093700004F001032021994041F007010246CDE7A6
:10938000A94BD6F8030000221A55A64B03EB840321
:109390001B6B9847A54B43F82400B078202100F0C0
:1093A0000102914041F0060153F8202046E604F006
:1093B0000101202606FA01F141F01001C9B260084E
:1093C00004F078F9C3B2AC780193EA7804F00101B3
:1093D00006FA01F1D20841F010010092C0F30743F0
:1093E0000022C9B2600804F0C3F803B0F0BD04F075
:1093F0000101202505FA01F141F01001C9B2600810
:1094000004F058F9B478F27804F0010105FA01F19A
:10941000D208C0F3072341F0100101920093DDE769
:1094200020F0020231E6202604F0010106FA01F1E3
:1094300041F01401C9B2600804F03CF9AB78D5F8EA
:10944000032003F0010106FA01F141F0140112B901
:1094500040F0010219E620F0010216E6202604F091
:10946000010106FA01F141F01401C9B2600804F0EB
:1094700021F9AB78D5F8032003F0010106FA01F1D8
:1094800041F0140112B140F01002FEE520F010028C
:10949000FBE5644BD6F8030003EB84031B6B984792
:1094A00004F001032021994041F0040166E750F8DF
:1094B0002430D5F8030098472021B94041F0050138
:1094C0000246C9B230462BE700EB8404D5F803000E
:1094D000236B98472021B94041F00801F0E7514B38
:1094E000D6F8030053F82430984704F001032021F4
:1094F000994041F0030141E74A4BD6F8030053F885
:109500002430984704F001032021994041F00B01D9
:1095100034E7444BD6F8030053F82430984704F05E
:1095200001032021994041F0120127E73D4BD5F876
:10953000030053F8243098472021B14041F0130133
:109540000246C9B23846EBE6202404FA06F141F09F
:109550001401C9B2384604F0ADF8AB78D5F8032051
:1095600003F0010104FA01F141F0140112B140F0DD
:1095700008028AE520F0080287E520F0040284E56D
:10958000202504F0010105FA01F141F01401C9B2EE
:10959000600804F08FF8B378D6F8032003F00101D7
:1095A00005FA01F141F0140112B140F400626CE5DA
:1095B00020F4006269E5D6F803102046C9B203B072
:1095C000BDE8F04004F07AB9D6F803102046C9B2DD
:1095D00003B0BDE8F04004F089B9210101F01001A9
:1095E00041F06E01600804F065F8B478F3780193F7
:1095F0002101C0F3072001F01001009000231A465A
:1096000041F06E01EEE6D6F80330022B3FF6CFAC08
:109610000448F378044484F84830E6E60894FF1FD1
:10962000EA93FF1F7886FF1F5096FF1F3896FF1F93
:10963000D6F80310C1F10801C9B2204603B0BDE855
:10964000F04004F00BB9D6F803102046C9B203B0BD
:10965000BDE8F04004F0D2B8D6F803102046C9B2F5
:1096600003B0BDE8F04004F059B9204604F05AFABE
:10967000D6F80310B378C9B228B9184603B0BDE8CC
:10968000F04004F0CBB9184603B0BDE8F04004F058
:109690008DB9204604F046FAD6F80310C9B228B9AD
:1096A000B07803B0BDE8F04004F090B8B07803B0F3
:1096B000BDE8F04004F09AB9D6F803102046C9B2CC
:1096C00003B0BDE8F04004F061B8D6F803102046BE
:1096D000C9B203B0BDE8F04004F08BBAD6F803106D
:1096E0002046C9B203B0BDE8F04004F09ABAD6F8FB
:1096F00003102046C9B203B0BDE8F04004F061BADF
:10970000D6F803102046C9B203B0BDE8F04004F01B
:10971000E5BAD6F803102046C9B203B0BDE8F04060
:1097200004F0B4B8D6F803102046C9B203B0BDE8BF
:10973000F04004F075B9454BD6F8030053F82430D7
:109740009847434B03EB841420614EE6D6F8031090
:109750002046C9B203B0BDE8F04004F0F7B8D6F82F
:1097600003102046C9B203B0BDE8F04004F05EB873
:10977000D6F803102046C9B203B0BDE8F04004F0AB
:1097800065BBD6F803102046C9B203B0BDE8F0406F
:1097900004F014BB2E48D6F8033000EB8414237277
:1097A00023E62A4BD6F8030053F824309847A40147
:1097B000274B185119E6254BD6F8030053F82430EF
:1097C0009847234B03EB841460600EE6204BD6F8D9
:1097D000032003EB84135A83204603B0BDE8F04016
:1097E00004F05ABDD6F80310204603B0BDE8F0409F
:1097F00004F018BE1648D6F8033000EB8414236238
:10980000F3E5D6F8033093B1012B7FF4D0AB104AC7
:109810000E4802EB841213760E4B40F8243000EB16
:1098200084040D4B23650D4B23630D4B0BE0084A5D
:10983000064802EB841213760A4B40F8243000EB02
:10984000840423652363A366CFE500BF7886FF1FEA
:109850000894FF1F79E10000F1E10000C1E1000080
:1098600039E2000069E20000F8B5CE4DCE4CA87890
:109870006B78052802D904232370F8BDA32B00F0D0
:109880008E8200F2C480112B00F0108258D8082B71
:1098900000F0C58128D8032B00F0748116D8012B65
:1098A00000F001054FEA500200F0678140F24D815F
:1098B000BE4B202103EB8000A94041F00701066D5B
:1098C000C9B2104603F0F6FEB04746E1052B00F0A2
:1098D0008481C0F07B81062B00F08781072B00F08C
:1098E00092810323237039E10C2B00F0B98112D847
:1098F0000A2B00F0A48140F29F8100F00103202197
:10990000994041F01501C9B2400803F0D3FEC043AD
:1099100000F0010021E10E2B00F0B081C0F0A78122
:109920000F2B00F0B881102BDBD1A04B03EB800391
:1099300020211D6D00F00103994041F005012BE14C
:109940001A2B00F0FD812DD8152B00F0CD8112D8F7
:10995000132B00F001064FEA5005944A4FEA8000AD
:1099600000F0BB8140F2AD8102442021B140176D6F
:1099700041F00B01ABE1172B00F0CA81C0F0BD81B3
:10998000182B00F0D081192BABD100F0010320215E
:10999000994041F01401C9B2400803F08BFEC0F3B6
:1099A0008000DAE0202B00F0E68116D81C2B00F0B6
:1099B000D781C0F0D2811D2B00F0D5811F2B90D113
:1099C00000F001032021994041F01001C9B2400884
:1099D00003F070FEC0F30340BFE07F2B00F0D581A1
:1099E0000CD8212B7FF47DAF010101F0100141F073
:1099F0006E01400803F05EFE0012AEE08C2B00F01A
:109A0000C981A22B7FF46DAF04F044F8A5E0B92B17
:109A100000F0128240D8AC2B00F0E2811FD8A72BB7
:109A200000F0D2810DD8A52B00F0BF8140F2BA81A1
:109A300004F078F8002840F0C381A87804F01EF8FC
:109A40008BE0A92B00F0C681C0F0C181AA2B00F0E9
:109A5000C481AB2B7FF445AF04F058F97DE0B32B04
:109A600000F0C7810AD8AE2B00F0C081C0F0BB81E6
:109A7000B12B7FF436AF04F031F86EE0B52B00F077
:109A8000C681C0F0B981B62B00F0CB81B82B7FF432
:109A900028AF04F053F860E0C92B00F0F0811CD827
:109AA000C12B00F0D2810BD8BC2B00F0C881BD2B9C
:109AB00000F0C881BB2B7FF414AF04F017FA4CE020
:109AC000C32B00F0CF81C0F0C581C42B00F0D3813F
:109AD000C52B7FF406AF364BCEE1D02B00F0E481EE
:109AE00023D8CC2B00F0D28107D8CA2B7FF4F9AE53
:109AF000304B03EB8010438BB0E0CE2B00F0C981DC
:109B0000CF2B7FF4EEAE2C4B195C0022626009B1C2
:109B1000012161601A54294B1A5C1AB1626842F043
:109B20000202626000221A5418E0D22B00F0C981B0
:109B3000C0F0C481D42B00F0D181FF2B7FF4D1AED3
:109B40001C4B03EB8010037E88E02021A94041F0EC
:109B50000D01C9B2104603F0ADFD6060184B1B78D3
:109B600053B1184B62681A60174B002A40F0BB8152
:109B70001A6842F008021A60F8BD2021A94041F09D
:109B80000101E6E7094B03EB800320211D6D00F086
:109B90000103994041F00201C9B2400803F08AFD77
:109BA000E7E000BF5896FF1F7098FF1F7886FF1FE1
:109BB0008C95FF1F0894FF1F0094FF1FE493FF1F65
:109BC0006B98FF1F5C98FF1F6096FF1FBF4B03EB56
:109BD0008000036D80699847BFE7BC4BBC4A03EB2C
:109BE000800352F820009B6EF5E700F0010320216E
:109BF000994041F01001C9B2400803F05BFDC0F389
:109C00000720C000A9E700F001032021994041F09E
:109C10001001C9B2400803F04DFDC0B2F1E700F0F9
:109C200001032021994041F01501C9B2400803F019
:109C300041FDC0F3402090E704F08CFA8DE700F07E
:109C400001032021994041F01501C9B2400803F0F9
:109C500031FD10F0020F0CBF0123002363607DE78C
:109C600000F001032021994041F01401EDE700F0DC
:109C700001032021994041F0140144E600F0010362
:109C80002021994041F01401C9B2400803F012FDAF
:109C9000C0F3001061E78D4B03EB800320219D6E24
:109CA00000F00103994041F0040175E7874B03EB95
:109CB000800320219D6E00F00103994041F00801CE
:109CC0006AE702442021B140976E41F00A01C9B20F
:109CD000284603F0EFFCB8473FE702442021B1409B
:109CE000176D41F00301F2E700F0010320219940D4
:109CF00041F00C01C9B240082DE7744B03EB80031F
:109D000020211D6D00F00103994041F0120143E74D
:109D10006E4B03EB800320211D6D00F00103994081
:109D200041F0130138E700F001032021994041F090
:109D30001401C9B2400803F0BDFCC0F3C0000CE739
:109D400000F001032021994041F01401C9B24008FC
:109D500003F0B0FCC0F3C020FFE603F0CBFEFCE64E
:109D600003F0D4FEF9E6594B03EB80031D6D02F0BE
:109D70008FFBA847F1E6010101F0100141F06E01EF
:109D8000400803F097FCC0B2E7E6504B184490F847
:109D9000483063E703F096FEC0F10800DDE603F00B
:109DA000C1FEDAE603F0D6FED7E603F0BBFE18B933
:109DB000A87803F0F8FED0E6A87803F0D7FECCE64A
:109DC000A87803F0E4FEC8E603F042FEC5E603F01F
:109DD000DDFFC2E603F0A6FFBFE603F0AFFFBCE67F
:109DE00003F0B8FFB9E603F0DDFFB6E603F0BEFF0F
:109DF000B3E603F0DAFEB0E6010101F0100141F034
:109E00006F01400803F056FCC0F30440A5E62F4A5A
:109E1000304B03EB801302EB8000026D1869904712
:109E20009BE62A4B03EB800320211D6D00F001030C
:109E3000994041F01101AFE603F038FE8DE604F0E1
:109E400061F88AE604F069F887E6224B03EB80109C
:109E5000037A03E71D4B1F49820103EB8000036D6A
:109E60008858B8E6194A1B4B03EB801302EB8000BD
:109E7000026D5868D3E7184B53F82030EEE600F037
:109E800001032021994041F0180133E704F00AF85A
:109E900063E6010101F0100141F06F01400803F099
:109EA00009FCC0F3090058E6010101F0100141F07E
:109EB0006F01400803F0FEFB00164EE604F0A8FA1E
:109EC0004BE6044B03EB8010C369C7E67886FF1F9F
:109ED0003896FF1F0894FF1FC493FF1F044B03EB2A
:109EE0008010036ABAE61A6822F0080243E600BF4F
:109EF0000894FF1F38B5C24A9378022B144600F02D
:109F00000881032B00F00C81002B40F0378253783E
:109F10004E2B00F0B48030D8462B00F0828012D84F
:109F2000422B6ED006D8402B5FD0412B64D0032249
:109F3000B44B58E0442B69D0452BF8D1B24BD178C3
:109F40005971052054E04B2B00F089800BD8472B2A
:109F50006FD0492BEBD1D278AB4B002A7AD1DA758E
:109F6000D97D172044E04C2B00F084804D2BDED1AE
:109F7000A54BD178597515203AE0542B00F0A680F6
:109F80001BD8512B00F08D8009D84F2B00F0828018
:109F9000502BCCD19C4BD1789975162028E0522BB0
:109FA00000F08C80532BC2D1974DD2F80330294654
:109FB000042241F8103F102043E0842B00F09E80E3
:109FC0000AD8552B00F08E80832BB0D18F4BD2F85E
:109FD0000320C3F8802038BD852B00F09480FF2B30
:109FE000A5D1D2788A4B1A7038BDD17845F2FF706E
:109FF000BDE83840FEF7BBBE834BD1781970002016
:10A00000F6E7814BD17859700120F1E77E49D2F80B
:10A01000033041F81C3F04221C20BDE83840FEF705
:10A02000B8BE7949D2F8033041F80C3F04220C2025
:10A03000F3E7754DD2F803302946042241F8083F72
:10A040000820FEF7A6FE2A8A29896879BDE83840EB
:10A0500003F03CB86B490122DA754A6080E76A4C2C
:10A06000D178E1700320FEF782FEE078BDE8384049
:10A07000FEF778BB644BD17899700220B8E7624C48
:10A08000D2F80300E084FEF773FD022204F12601FA
:10A090002620C2E7D2F803105B4BC9B259761920CB
:10A0A000A6E7594D2A7DD20704D5E378DB0701D412
:10A0B000FEF7C6FEE1782975142099E75249D2F8D7
:10A0C000033041F8203F04222020A6E7D2F80330D5
:10A0D000012B00F253814C49D37801F81A3F012239
:10A0E0001A209AE7D2F80330012B00F24781464943
:10A0F000D37801F81B3F01221B208EE7454BD2F895
:10A1000003201A6038BD414BD2F80320C3F88420E5
:10A1100038BD5178404BD2F8032043F8212038BD98
:10A1200053782E2B3FF603AF01A252F823F000BF65
:10A13000EDA1000021A2000035A200002F9F000029
:10A140002F9F00002F9F00002F9F00002F9F0000D7
:10A150002F9F000049A2000053A200005DA2000052
:10A1600067A2000071A200007BA200002F9F0000E8
:10A170002F9F00002F9F00002F9F00002F9F0000A7
:10A180002F9F00002F9F00002F9F00002F9F000097
:10A190002F9F00002F9F00002F9F000085A200002E
:10A1A00093A20000A1A20000AFA20000BDA2000087
:10A1B000CBA20000D9A20000E7A20000F5A2000097
:10A1C00003A3000011A300001FA300002DA30000A3
:10A1D00037A3000041A300004BA3000055A30000DB
:10A1E0005FA3000069A3000073A300000B4BD4F829
:10A1F00003201A60FEF740FA044BC3F8880038BD0C
:10A200005896FF1F7098FF1F0C80FF1F7886FF1F56
:10A210006A98FF1F6C98FF1F7C98FF1FA495FF1F73
:10A22000574BD4F803205A60FEF726FA554BC3F873
:10A230008C0038BD524BD4F803209A60FEF71CFA0C
:10A24000504BC3F8900038BD4D4BD4F80320DA6072
:10A2500038BD4B4BD4F803201A6138BD484BD4F8B5
:10A2600003205A6138BD464BD4F803209A6138BDAB
:10A27000434BD4F80320DA6138BD414BD4F80320B6
:10A280001A6238BDD4F803303D4ADBB282F824307C
:10A2900038BDD4F803303A4ADBB282F82A3038BDF0
:10A2A000D4F80330364ADBB282F8253038BDD4F812
:10A2B0000330334ADBB282F82B3038BDD4F8033098
:10A2C0002F4ADBB282F8263038BDD4F803302C4A4E
:10A2D000DBB282F82C3038BDD4F80330284ADBB228
:10A2E00082F8273038BDD4F80330254ADBB282F833
:10A2F0002D3038BDD4F80330214ADBB282F8283043
:10A3000038BDD4F803301E4ADBB282F82E3038BD97
:10A31000D4F803301A4ADBB282F8293038BDD4F8B9
:10A320000330174ADBB282F82F3038BD144BD4F813
:10A3300003201A6338BD124BD4F803205A6338BD8A
:10A340000F4BD4F803209A6338BD0D4BD4F803208B
:10A35000DA6338BD0A4BD4F803201A6438BD084BC1
:10A36000D4F803205A6438BD054BD4F803209A640E
:10A3700038BD034BD4F80320DA6438BD0422D7E596
:10A38000A495FF1F7886FF1F2DE9FF47C74EC84FD2
:10A3900032787A7064233B70212AD6F803307B60D0
:10A3A00034463D4601F0CA8000F2C7800E2A00F014
:10A3B000548539D8072A00F0EE8314D8032A00F018
:10A3C000518208D8012A00F0A081022A00F0F6810B
:10A3D00002232B70DEE1052A00F0DA8340F26C8262
:10A3E000FFF742FAD6E10A2A00F0DB8307D8082AF1
:10A3F00000F0D483092AEBD1FFF77CFDCAE10C2AD7
:10A4000000F0FE8440F2E784B078052800F2D381A2
:10A410007378012B00F00985C0F00485022B00F051
:10A42000078503233B70B5E1182A00F0658630D814
:10A43000142A00F0AB8515D80F2A00F02985132ABD
:10A44000C6D171789B4A092900F27685DFE811F0C0
:10A4500071057C057F05820586058D0590059305B0
:10A4600096058B05162A00F0428640F2B085924A86
:10A47000D2F89C10072900F28D81481C02EB810163
:10A48000C2F89C00D2F89800C1F8A000C2F8983039
:10A4900080E11C2A00F0558722D81A2A00F04E8647
:10A4A00040F23B86844D95F8C12072B95E1C04BF12
:10A4B000804B1B680A205843C5F8C400FEF7DCF83F
:10A4C0000123C5F8C80085F8C1306378042B00F279
:10A4D0006181DFE813F044069106C806FF065C06BA
:10A4E0001F2A00F0648700F2B5871E2A7FF470AF40
:10A4F0007278142A00F27E84B678052E00F227873F
:10A5000006206E4C00FB026144F821306C4B9B7EB0
:10A51000002B00F03F81002A00F03C8110FB02611B
:10A520001820013A424302F5D360042204EB810172
:10A5300002FB0600FEF72DFC2CE1802A01F0DB80F7
:10A5400044D8402A01F0BF8029D8242A01F0548041
:10A550000CD8222A01F04880232A7FF439AF554BCA
:10A560001B68C6F80330FFF7C5FC13E1262A01F08B
:10A570008180C1F07480272A7FF42AAFB278052A3F
:10A5800000F219817378142B00F23484062101FB48
:10A590000323484A1168494A42F82310FAE0442A42
:10A5A00001F09D8007D8422A01F0958041F28F800A
:10A5B00001F069FFEEE0462A01F09980C1F0938036
:10A5C000472A7FF405AF01F062FFE3E0872A01F03C
:10A5D000408146D8832A01F0AD800AD8812A01F053
:10A5E0009080822A7FF4F4AE334B022283F89420C9
:10A5F000D0E0852A01F0D380314A41F2BD80314953
:10A60000314C01250D70B3F5C05F9178217081F058
:10A61000CC80127D12EA050641F0C780184602A9D7
:10A62000FEF707FC9DF8083063709DF80930A370B1
:10A630009DF80A30E3709DF80E3023719DF80D30BF
:10A6400063719DF80C30A3719DF80B30E371267295
:10A650002B46E15C227A01330A44082B2272F8D19E
:10A6600098E08C2A01F03E813CD8892A01F01F81B4
:10A67000C1F0A5808A2A7FF4ABAE7278134B002A12
:10A6800041F02D811A70124AE37813700A4A92F849
:10A69000B011104A1170104900220A700F490A7057
:10A6A0000F4A11780B43137074E000BF5896FF1FD8
:10A6B0007098FF1F5C98FF1F7886FF1F6496FF1F2E
:10A6C0000C80FF1F6098FF1F6198FF1FDC93FF1F26
:10A6D000F193FF1F0796FF1FF093FF1F5696FF1F72
:10A6E000DD93FF1FF22A01F06C81FF2A01F0AE8199
:10A6F0008D2A7FF46DAE7278032A01F25E81DFE865
:10A7000012F0310918094A095809B078052852D8B9
:10A71000964B974E00251D54964B1D54335C73B1D8
:10A7200000F0010320219940934B41F0060153F8BA
:10A730002020C9B2400802F075FFA378F554A6782E
:10A740008E4BD4F8030001279F558D4B002853F8FA
:10A750002630B8BF40429847202506EA070105FA8F
:10A7600001F141F007010246C9B226FA07F002F0F2
:10A7700059FFD4F80330A078002B0EDD00EA070162
:10A78000002305FA01F1019700931A46C9B2F84077
:10A7900002F0EEFE04B0BDE8F08700F001010223F4
:10A7A00005FA01F10193002300931A46C9B240084B
:10A7B00002F0DEFEEEE704232B70EBE7B07805280D
:10A7C000F9D86A4B6A4E00251D546A4B1D54335C00
:10A7D00073B100F0010320219940674B41F006015D
:10A7E00053F82020C9B2400802F01CFFA378F554AA
:10A7F000A678624BD4F8030001279F55604B0028D0
:10A8000053F82630B8BF40429847202506EA070192
:10A8100005FA01F141F007010246C9B226FA07F034
:10A8200002F000FFD4F80330A078002B0DDD00EA21
:10A830000701022305FA01F10193002300931A4650
:10A84000C9B2F84002F094FEA4E700F00101002331
:10A8500005FA01F1019700931A46C9B2400802F0C7
:10A8600087FE97E7B0780528A5D802F06DFBB07891
:10A87000424B012200EA0201202404FA01F141F0D6
:10A8800007011A54C9B20022400802F0CBFEB0788A
:10A8900000F0010104FA01F1022300240193224691
:10A8A00023460094C9B2400802F062FEB3782F4AF2
:10A8B000D454304AD4546DE7B078052803D972785F
:10A8C000022A7FF467AF294A00261654294A1654F3
:10A8D0006278012A56D005D3022A00F0BB800323F8
:10A8E0002B7057E7254D2B5C7BB1254B00F0010207
:10A8F000202103EB8003914041F007019A69C9B21E
:10A90000400802F08FFEA378EE54A078184D2B5C1F
:10A910007BB100F0010320219940174B41F0060163
:10A9200053F82020C9B2400802F07CFEA378002230
:10A93000EA54A078D4F80320202500F0010105FA9C
:10A9400001F141F00D01C9B2400802F06BFEA078A0
:10A9500000F00101002305FA01F1019300931A466A
:10A96000C9B2400802F004FE14E700BFE493FF1FE1
:10A970005096FF1F0094FF1F3896FF1FEA93FF1F9A
:10A980007886FF1FB54F3B18202193F84830012BE4
:10A9900057D04BD3022B5AD0A078DFF8CC8218F8CE
:10A9A000003083B100F001032021994007EB8007BC
:10A9B00041F00701BA69C9B2400802F033FEA3783A
:10A9C000002208F80320A078A54F3B5C7BB100F083
:10A9D000010320219940A34B41F0060153F82020A8
:10A9E000C9B2400802F01EFEA3780022FA54A078F3
:10A9F000D4F8033000F00101202707FA01F11E44CA
:10AA000041F00D013246C9B2400802F00BFEA078B9
:10AA100000F00101002307FA01F1019300931A46A7
:10AA2000C9B2400802F0A4FD6E60B3E600F0010375
:10AA3000994041F00D01C9B2400802F03BFE0646C4
:10AA4000AAE700F00103994041F00101F3E703F0A8
:10AA5000DFFCF4E7142B3FF7AEAE02064CD5824F75
:10AA6000DFF8FC81DFF808923546A3782B41DB073D
:10AA70003ED5EB5D05F0010A6E086BB120217B4BE2
:10AA800001FA0AF141F0070153F82520C9B2F0B2EA
:10AA900002F0C8FD0023EB5515F8083073B12021F2
:10AAA000704B01FA0AF141F0060153F82520C9B2B2
:10AAB000F0B202F0B7FD002305F80830202303FAB6
:10AAC0000AFAD4F80330062202FB0353F6B24AF026
:10AAD0000D0159F82320C9B2304602F0A3FD00232E
:10AAE000019300931A465FFA8AF1304602F040FD66
:10AAF0000135062DB9D14DE605283FF65CAE5A4D1D
:10AB00002B5C7BB1554B00F00102202103EB80034D
:10AB1000914041F007019A69C9B2400802F082FDF4
:10AB2000A378EE54A0784E4D2B5C7BB100F001036E
:10AB3000202199404B4B41F0060153F82020C9B227
:10AB4000400802F06FFDA3780022EA54A078D4F800
:10AB500003302025062200F0010102FB030305FA61
:10AB600001F1434A41F00D0152F82320C9B24008D7
:10AB700002F058FDA07800F00101002305FA01F170
:10AB8000019300931A46C9B2400802F0F1FC01E6B5
:10AB9000FEF706FAFEE5FEF7F5F9FBE5FEF7F2F93A
:10ABA000F8E5B378022B00F0CA80032B00F0CC80CC
:10ABB000002B40F009817378502B00F0928024D84C
:10ABC000472B7ED011D8422B72D006D8402B55D0BF
:10ABD000412B69D003232B7055E0452B6BD06DD8EA
:10ABE000442BF7D1234BDB6960E04C2B72D006D8A5
:10ABF000492B69D04B2BEDD11E4BDB7856E04E2B09
:10AC00001C4B6CD069D95B7E50E0802B78D012D879
:10AC1000532B6CD006D8512B66D0522BDAD1154B62
:10AC20001B6A43E0552B68D064D3562BD2D1114B0D
:10AC300093F824303AE0832B6DD007D8812B63D072
:10AC4000822BC7D1054BD3F898302FE0852B69D0E4
:10AC500065D3FF2BBED1084B1B7837E07886FF1FEA
:10AC60005096FF1F3896FF1FEA93FF1F9086FF1F25
:10AC70006496FF1F0C80FF1F6A98FF1F45F2FF704C
:10AC8000FEF7AEF87860994B1B78002B3FF482AD4D
:10AC9000974B6A681A60974B002A40F097801A68B1
:10ACA00042F008021A6075E5934B1B786B60EAE787
:10ACB000914B5B78FAE7904B5B79F7E78E4BDB685B
:10ACC000F4E78D4B9B68F1E78B4BDB7D003318BFBE
:10ACD0000123EBE7884B9B78E8E75B7DE6E7DB8CBD
:10ACE000E4E7854B9B7DE1E7834B1B7DDEE7824BF1
:10ACF0001B69DBE7804B9B7ED8E77F4BDB7ED5E78C
:10AD00007E4B93F89430D1E77C4B93F894301E1F20
:10AD100073427341CAE7794BD3F88030C6E7784B6A
:10AD20001B68C3E7754A7748D2F8843043F239018B
:10AD300000FB0313C2F8843023F00043B6E77278B7
:10AD4000714B53F82230B1E77378282B2DD014D8EB
:10AD5000022B28D006D823B3012B7FF43BAF6B4BDB
:10AD60005B68A3E7092BFFF435AF0E2B8BD9272B9C
:10AD70007FF430AF654B1B6B98E72B2B1BD007D8AC
:10AD8000292B15D02A2B7FF425AF604BDB6B8DE789
:10AD90002D2B16D012D32E2B7FF41CAF5B4BDB6C0C
:10ADA00084E75A4BBCE7594B8CE7584B5B6B7DE70C
:10ADB000564B9B6B7AE7554B1B6C77E7534B5B6CA1
:10ADC00074E7524B9B6C71E7042304E71A6822F086
:10ADD00008021A60DEE4B378022B0ED170783728AF
:10ADE00008D800F5FF704A49800004220144FDF7AD
:10ADF000D0FFCFE403232B70CCE404233B70C9E4E1
:10AE0000B378022B0BD170783728F3D800F5FF7098
:10AE10003F49800004220144FDF7F4FFBAE4042313
:10AE20003B70B7E402F088F8B4E402F08DF8B1E4C6
:10AE300002F092F82D4B78601B78002B3FF4AAACFF
:10AE40002B4B18602B4B1A6818B942F008021A6095
:10AE5000A0E422F008021A609CE4B278022A14D11D
:10AE60007078072806D813B9FDF7C8FD92E4FDF7FE
:10AE7000B1FD8FE4FF287FF48DAC5D1C0ABF1C4B35
:10AE8000D8B21878FDF7CEFD84E404233B7081E44A
:10AE9000B378012B40D023B1022B41D004233B7067
:10AEA0000FE07078082803D8FDF7CDFD686008E052
:10AEB0000A2815D1174B1B6983F40073C3F3402391
:10AEC0007B600A4B1B78002B3FF464AC084B6A682C
:10AED0001A60084B42BB1A6842F008021A6059E433
:10AEE000FF28EED1FDF7E6FDE0E700BF6B98FF1FFE
:10AEF0005C98FF1F6096FF1F0C80FF1F7886FF1F66
:10AF00006C98FF1F6D4EC6417C98FF1FA495FF1FD4
:10AF10008490FF1F80F00F40707802F0A7F8C5E71B
:10AF20007078FDF7A9FDC1E71A6822F008021A60DF
:10AF300030E41068184410601268AB4B0ABB1A6802
:10AF400042F008021A6025E41068C01AF3E710689E
:10AF50005843F0E7106890FBF3F0ECE7116891FBC1
:10AF6000F3F003FB10131360E6E710681840E2E704
:10AF700010681843DFE710685840DCE71368DB43CC
:10AF8000F1E71A6822F008021A6003E4974A116890
:10AF9000954A8B4213680BDA23F0030343F0040352
:10AFA0001360136871B943F008031360FFF7F2BB35
:10AFB0000BBF23F0060323F0050343F0010343F026
:10AFC0000203EDE723F008031360FFF7E3BB727899
:10AFD0000C2A3FF6DFABDFE802F007111B252F3903
:10AFE000444E58626C7680007F4A126814077FF5E1
:10AFF000D1AB7F4AC2F89830FFF7CCBB7A4A1268CF
:10B0000010073FF5C7AB7A4AC2F89830FFF7C2BBCA
:10B01000754A1268D1077FF5BDAB754AC2F8983002
:10B02000FFF7B8BB704A1268D2073FF5B3AB704A5E
:10B03000C2F89830FFF7AEBB6B4A126857077FF52E
:10B04000A9AB6B4AC2F89830FFF7A4BB664A1268F6
:10B0500012F0050F3FF49EAB654AC2F89830FFF737
:10B0600099BB614A126896077FF594AB604AC2F8B3
:10B070009830FFF78FBB5C4A126895073FF48AABA4
:10B080005B4AC2F89830FFF785BB574A1268D4066E
:10B090007FF580AB564AC2F89830FFF77BBB524A27
:10B0A000126890067FF576AB514AC2F89830FFF7E8
:10B0B00071BB4D4A126851067FF56CAB4C4AC2F821
:10B0C0009830FFF767BB484A126812067FF562ABFB
:10B0D000474AC2F89830FFF75DBB434A1268D7056C
:10B0E0007FF558AB424AC2F89830FFF753BB404A4D
:10B0F000C2F89830FFF74EBB3D4AD2F89C30002B87
:10B100003FF448AB013BC2F89C3002EB8303D3F819
:10B11000A030C2F89830FFF73DBB73782E2B04D8CF
:10B12000344A0121D154FFF735BBFF2B7FF462AEC7
:10B130002F4B012283F8C020FFF72CBB73782E2BF6
:10B1400004D82C4A0021D154FFF724BBFF2B7FF4F5
:10B1500051AE274B002283F8C020FFF71BBBFDF741
:10B160008BFAD5F8C830C01A0028D5F8C430B8BF5B
:10B170004042984295BFD5F89830002303F1FF3341
:10B1800085F8C13098BFC5F89830FFF703BBA078A9
:10B1900001F0E2FE40B9144A85F8C100136823F0BB
:10B1A00010031360FFF7F6BAD5F8C430ABB1FDF762
:10B1B00063FAD5F8C830C01A0028D5F8C430B8BF33
:10B1C0004042984209D9084A002385F8C1301368E3
:10B1D00043F010031360FFF7DDBAD5F89830013B58
:10B1E000C5F89830FFF7D6BA6096FF1F5C98FF1F2E
:10B1F0007886FF1F0896FF1FA078202100F001032A
:10B20000994041F01501C9B2400802F053FA10F418
:10B21000007409D0C34A002385F8C130136823F0B5
:10B2200010031360FFF7B6BAD5F8C430A3B1FDF729
:10B2300023FAD5F8C830C01A0028D5F8C430B8BFF2
:10B240004042984208D9B74A85F8C140136843F094
:10B2500010031360FFF79EBAD5F89830013BC5F88C
:10B260009830FFF797BAA078202100F001039940A9
:10B2700041F01501C9B2400802F01CFA10F00104B7
:10B2800009D0A84A002385F8C130136823F01003C1
:10B290001360FFF77FBAD5F8C430A3B1FDF7ECF91E
:10B2A000D5F8C830C01A0028D5F8C430B8BF40421D
:10B2B000984208D99B4A85F8C140136843F01003AF
:10B2C0001360FFF767BAD5F89830013BC5F898309E
:10B2D000FFF760BAA078202100F00103994041F007
:10B2E0001501C9B2400802F0E5F910F0020409D0D6
:10B2F0008C4A002385F8C130136823F010031360D3
:10B30000FFF748BAD5F8C430A3B1FDF7B5F9D5F8C1
:10B31000C830C01A0028D5F8C430B8BF404298429F
:10B3200008D9804A85F8C140136843F010031360C0
:10B33000FFF730BAD5F89830013BC5F89830FFF7E1
:10B3400029BA794B002283F89420FFF723BAFF2E05
:10B350007FF431AA754E42B300254FF00608182736
:10B36000607818FB00510138784300F5D36000EB9A
:10B370008500042206EB81010135FDF70AFD062D4B
:10B38000EED1FFF707BA6119781904223144043568
:10B39000FDF7FFFC182DF6D11834B4F5FC7F3FF40F
:10B3A000F9A9002504F5D067EDE71824F9E77378CB
:10B3B000142B3FF61FADB278052A1BD8062101FBDE
:10B3C00003235A4A52F82320594B7A601B78002BEA
:10B3D0003FF4E0A9574B1A60524B2AB91A6842F061
:10B3E00008021A60FFF7D6B91A6822F008021A603C
:10B3F000FFF7D0B9FF2A7FF4DEA94C4E43B30025F6
:10B400004FF006081827607818FB00510138784380
:10B4100000F5D36000EB8500042206EB81010135C5
:10B42000FDF7F0FC062DEED1FFF7B4B961197819DC
:10B43000042231440435FDF7E5FC182DF6D118340B
:10B44000B4F5FC7F3FF4A6A9002504F5D067EDE72D
:10B450001824F9E77778142F3FF6CCACB67830068D
:10B4600032D5324E344F00254FF02008A3782B41BF
:10B47000D90711D505F0010108FA01F141F00101E8
:10B4800094F80190C9B2C5F3470002F013F90623FE
:10B4900003FB095946F82900BB7E83B1637873B179
:10B4A000062111FB03511820013B584300F5D360DE
:10B4B000042206EB810100EB8500FDF76AFC0135F3
:10B4C000062DD3D1FFF766B9052E3FF674A906F015
:10B4D00001032021994041F001017008C9B202F036
:10B4E000E9F8154B114D9B7E062202FB076645F8D5
:10B4F0002600002B3FF44EA96378002B3FF44AA9A5
:10B50000A07812FB03015A1E1823534303F5D3639B
:10B51000042205EB810102FB0030FDF73AFCFFF746
:10B5200039B900BF6096FF1F7886FF1F6496FF1F22
:10B530006B98FF1F5C98FF1F0C80FF1F7278AE4B4B
:10B540000A2A0CD8DFE802F006151A1F252D32371B
:10B550003C414500A9491A6809680A441A601A68FA
:10B56000A74B002A3AD11A6842F008021A60FFF786
:10B5700011B9A2491A680968521AEFE79F4A196877
:10B5800012684A43EAE79D491A68096892FBF1F29A
:10B59000E4E79A4A1868116890FBF1F201FB120285
:10B5A000DCE796491A6809680A40D7E793491A68A0
:10B5B00009680A43D2E791491A6809684A40CDE709
:10B5C0008E490A68D2430A60C9E719688B4A11603C
:10B5D000C5E78A4A196810681860F8E71A6822F007
:10B5E00008021A60FFF7D6B8834B1B68C6F8033011
:10B5F000FDF7D6FCFFF7CEB87378052B3FF6CAA847
:10B60000DFE803F0030A11181F267D4A136803F0D0
:10B610000F031360FFF7BEB8794A136823F01003D5
:10B620001360FFF7B7B8764A136823F0200313605E
:10B63000FFF7B0B8724A136823F040031360FFF7B6
:10B64000A9B86F4A136823F080031360FFF7A2B80C
:10B650006B4A136823F480731360FFF79BB871780B
:10B660002E293FF6C7AB674A02EB8102C2F8CC3005
:10B67000FFF790B8634B604AD3F8881111605F4AB6
:10B68000D3F88C111160D3F89021C3F898205C4A4C
:10B69000D3F894111160D3F8982183F8C120D3F81E
:10B6A0009C21C3F8C820D3F8A021C3F8C42093F884
:10B6B000A411554A505C08B101205054002283F86F
:10B6C000A821FFF767B800F0DBFEFFF763B800F0D2
:10B6D000D8FEFFF75FB800F0D5FEFFF75BB800F0CB
:10B6E000D3FEFFF757B800F0D0FEFFF753B800F0D5
:10B6F000CDFEFFF74FB8434B002283F89420FFF7AD
:10B7000049B872782AB1012A09D003233B70FFF7A8
:10B7100041B83C4B012283F89420FFF73BB8B3F5C6
:10B72000C05FBFF448A8374981F89420C1F8983029
:10B73000FFF730B8334A3448002382F8C03082F82B
:10B74000A83102F1CC044FF0FF35194644F82350DC
:10B75000C15401332F2BF9D1274B82F89410196073
:10B76000264BC2F898101960254BC2F89C1082F83D
:10B77000C1101960FFF70EB8127D92070BD4B3F514
:10B78000C05FBFF418A81F4A042182F89410C2F8C1
:10B79000AC31FEF7FFBF08233B70FEF7FBBF194B30
:10B7A000002283F89420FEF7F5BF2B460022E254D6
:10B7B0000133082BFBD123782372FEF7EBBF73789C
:10B7C000012B2BD005D3022B31D003233B70FEF786
:10B7D000E1BF0E4B01221A700D4B0E4A9B7813707D
:10B7E0000D4B196800230139013311F8010FD054B2
:10B7F000082BF9D1FEF7CEBF5C98FF1F7898FF1F8A
:10B800006096FF1F7886FF1F0896FF1F6098FF1F36
:10B810000C80FF1F6198FF1F0880FF1F1822FA711C
:10B820007B7142220723BA713B71FEF7B3BF8D4B88
:10B830008D4801221A708D4B8D4A9B78137000231E
:10B8400001331918082B11F8091CD154F8D1FEF74F
:10B85000A1BF7378032B3EF69DAFDFE803F0021023
:10B860001E23844B93F89420FA7193F8C120D3F8E7
:10B87000AC31BA711A0A7A713B71FEF78BBF7D4BFE
:10B8800093F89420FA7193F8C120D3F89830BA71E4
:10B890001A0A7A713B71FEF77DBF774B1B687B609C
:10B8A000FEF778BF754B1B687B60FEF773BF72783D
:10B8B000002A7EF46FAFB17800297EF46BAF40F2BE
:10B8C000D24293427EF466AF45F2FF70FDF74FFA25
:10B8D000FDF7B6FA0120FCF7ABFFFEF75BBF0122D4
:10B8E000FEF7D0BE74782CB1012C13D003233B702B
:10B8F000FEF750BF042202A945F2FB70FDF782FA61
:10B90000029BD6F803209A4206BF01237B607C602D
:10B91000FEF740BFB3782A2B07D10422584945F2DD
:10B92000FB70FDF736FAFEF735BF03233B70FEF7D9
:10B9300031BF504CD4F8B401002104F5DC728142CF
:10B940003EF428AF52F821509D4201F1010520D16B
:10B9500002EB8503043B0138814214D3C4F8B401DF
:10B96000FEF718BF434AD2F8B41109299DBF481CFD
:10B97000C2F8B40102EB8102092394BFC2F8B831C6
:10B980003B70FEF707BF53F8042F43F8042C013136
:10B99000E2E72946D3E7374A0023C2F8B431194613
:10B9A00002F5DC7242F8231001330A2BFAD1FEF7BC
:10B9B000F1BE0A237B60FEF7EDBE03233B70FEF76A
:10B9C000E9BE7378812B7EF4F6AEB378922B7EF4C9
:10B9D000F2AEB379A32B7EF4EEAE7379B42B7EF482
:10B9E000EAAE3379C52B7EF4E6AEF378D62B7EF43F
:10B9F000E2AEFDF7F8F8FCF73FFE0446FCF73CFE2C
:10BA0000001B0028B8BF4042B0F57A7FF6DBFCF798
:10BA10000DFF1C4B00221A604FF0FF32C3F870215B
:10BA2000C3F87022C3F87421C3F87422C3F87821D4
:10BA3000C3F87822C3F87C21C3F87C22124B134A46
:10BA40001A600120FCF7F4FEFEF7A4BE40F2D242D9
:10BA500093427EF49FAE074B012283F8E021FEF76C
:10BA600099BE00BF6098FF1F008000000C80FF1F80
:10BA70006198FF1F7886FF1F5C98FF1F7898FF1F53
:10BA80005B96FF1F10E000E00080FF1F7856341225
:10BA90002DE9F84F484B494F00241C60484BC7F82C
:10BAA00098401C60474B87F8C1401C6007F1500963
:10BAB00007F1300A444B454A03EB84134FEA8408EC
:10BAC0001B7E002B45D1424B47F8243049F82430E7
:10BAD0004AF8243004F0010120268E4076B2C4F3E7
:10BAE000470B46F0070142F82430C9B2584601F02E
:10BAF000E1FD384A42F80800374A002546F00601C1
:10BB0000A554C9B2584601F0D5FD344B43F808009E
:10BB1000334BE0B2E554013402F0BEFB062CC9D130
:10BB2000304A2B462946904642F823100133B3F59C
:10BB3000807FF9D12C4EB37E43BBF37E53B3737D2C
:10BB4000BBB3FCF7FBFFA0B3012387F89430BDE83B
:10BB5000F88F264B47F82430254B49F82430254BE5
:10BB60004AF82430244BB5E7291909EB05000422D3
:10BB700051440435FDF746F9182DF5D11834B4F5C4
:10BB8000FC7FDAD0002504F5D069EDE71824DFF852
:10BB90006CA0F7E74FF4FF6440F6D805A4F5FF6109
:10BBA0002046042241440434FDF72CF9AC42F5D17F
:10BBB000C5E70023C9E700BF5C98FF1F7886FF1F19
:10BBC0007898FF1F6096FF1F0894FF1FE086FF1FF5
:10BBD00069E200009086FF1FEA93FF1F3896FF1F5F
:10BBE0005096FF1F7C98FF1F0C80FF1F79E100001B
:10BBF000F1E10000C1E1000039E200006496FF1F9E
:10BC0000F7B50F4C07460E4694E803008DE8030095
:10BC10000C49C1F803300C4B8A7000220F704E7033
:10BC20001A70FEF7B1FB094A217882F8E1119DE80C
:10BC30000300636884E80300184603B0F0BD00BF4A
:10BC40007098FF1F5896FF1F6B98FF1F7886FF1F85
:10BC5000F7B504461F4A63781370A3785370E378EE
:10BC600093702379937163795371A3791A4D13718A
:10BC7000E379D3700E4695E80300184B00221A7042
:10BC80008DE80300FEF780FB154B1A786F462B46B4
:10BC90009AB9327072702A78B2706A78F270EA7962
:10BCA0003271AA7972716A79B2712A79F27197E860
:10BCB000030083E8030003B0F0BD012AF7D109486F
:10BCC000721EF11D10F8014F02F8014F8A42F9D19E
:10BCD000EDE700BF5896FF1F7098FF1F6B98FF1F7E
:10BCE0006098FF1F6198FF1F014B93F8E1017047B7
:10BCF0007886FF1F2DE9F043994B9A4C1B788FB043
:10BD00006BB1994B1B78063BDBB2192B04D8974AD1
:10BD100022FA03F3D90702D4002384F8B03194F84F
:10BD2000B031934E5A1E012A51D89249012BCA684C
:10BD3000079214BF082307238DF81830327894F83F
:10BD4000E2318DF8193000238DF81A30002A33D1F2
:10BD50008B688DF82030884B8DF8272019788DF866
:10BD6000211059788DF82210D9798DF823109979FE
:10BD70008DF8241059791B798DF825108DF826300F
:10BD800006A801F091FA002800F02A837B4B1A786C
:10BD90009846002A00F01E81794B7A4F1B78013BB0
:10BDA000062B00F21381DFE813F0F100F1005801D7
:10BDB0001101110111017F01012AE1D17248013302
:10BDC00006AA1A44195CD171082BF8D1D8E7032BC5
:10BDD0003DD1337883BBDFF89C81674F98F8020030
:10BDE00098F801503B7805441D447B781D44FB794D
:10BDF0001D44BB791D447B791D443B791D44FCF7F0
:10BE000075FC98F80100FCF771FC3878FCF76EFCC3
:10BE10007878FCF76BFCF879FCF768FCB879FCF7EC
:10BE200065FC7879FCF762FC3879EDB2FCF75EFCD2
:10BE30002846FCF75BFCA9E7012BA7D1524F002550
:10BE4000785D0135FCF752FC092DF9D19EE7042BF2
:10BE50002BD1484FDFF82081B8787D78002301226C
:10BE60000544154488F8013088F80020C8F80430EB
:10BE7000FCF73CFC7878FCF739FC98F80000FCF7FC
:10BE800035FC98F80100FCF731FC98F80700FCF746
:10BE90002DFC98F80600FCF729FC98F80500FCF743
:10BEA00025FCEDB298F80400C0E7072B37D13378B2
:10BEB00053BB304B9F7893F801802F4B8DF8007067
:10BEC0001D785878D9798DF8025047443D449A79C5
:10BED0008DF80300284493F805C08DF80410014440
:10BEE00093F804E08DF805200A440CEB0203734438
:10BEF0008DF801808DF806C08DF807E08DF80830C8
:10BF00006846FCF76DFE41E7012BF9D11E4900237D
:10BF10005A5C0DF803200133092BF9D1F0E7082B07
:10BF20007FF434AF144A134900230120537010707A
:10BF300053608A7849788DF800200A4402448DF8CD
:10BF400001108DF802008DF803308DF804308DF863
:10BF500005308DF806308DF807308DF80820CFE7D2
:10BF60006A98FF1F7886FF1F5896FF1F1102000274
:10BF70006098FF1F0C80FF1F7098FF1F5696FF1FD1
:10BF80000796FF1FF093FF1F6198FF1FB24A397891
:10BF900093688DF8303080238DF831308A238DF806
:10BFA000323000238DF833308DF834308DF8353051
:10BFB0008DF836108DF8293007218DF82A300AA81F
:10BFC000D3688DF828100B9301F06EF900233B70B5
:10BFD00088F80030002384F8B031337094F8E031F1
:10BFE00013B10120FCF724FC06A801F0E9F806468D
:10BFF000002800F04981994B9DF820201A709DF887
:10C0000021205A709DF822209A709DF823209A7161
:10C010009DF824205A719DF825201A719DF826203C
:10C02000DA709DF8193084F8E231FCF725FB8C4B6F
:10C0300018608C4B00221A709DF81830072B0CBF2B
:10C040000123022384F8B03194F894305A1E012A57
:10C050004AD9052B48D0012247E0DFF8FC913B7814
:10C0600099F8020099F8015005440A351D44FCF77F
:10C070003DFB99F80100FCF739FB8020FCF736FB0B
:10C080008A20FCF733FB0020FCF730FB0020FCF794
:10C090002DFB0020FCF72AFBEDB23878FCF726FBDD
:10C0A0002846FCF723FB91E76B4A507893788DF88C
:10C0B0000C303A788DF80D00802103448DF80E1075
:10C0C0000A338A218DF80F101344002103A88DF83C
:10C0D00010108DF811108DF812108DF813208DF8B6
:10C0E0001430FCF77DFD71E700225F4B1A7094F865
:10C0F0009430042B04D1594B19780A0640F173810E
:10C1000094F8B021082A04D840F25113D340DF0735
:10C1100001D4FEF739F994F8B031092B77D1FCF747
:10C12000ABFAD4F88830514DC01A00282A68B8BF3D
:10C130004042904209D94E4B1A78012A04BF02228C
:10C140001A70FCF799FAC4F88800FCF795FAD4F84D
:10C150008C306A68C01A0028B8BF4042904209D9A2
:10C16000434B5A78012A04BF02225A70FCF784FA22
:10C17000C4F88C00FCF780FAD4F89030AA68C01A92
:10C180000028B8BF4042904209D9394B9A78012A19
:10C1900004BF02229A70FCF76FFAC4F8900094F87A
:10C1A000C030A3B394F8A8318BBB314A31481D4647
:10C1B000D15C022940F00B8150F823104E1C00F096
:10C1C00005812D4A84F8A4311268C4F888212B4ACD
:10C1D0001268C4F88C21D4F89820C4F89021284A19
:10C1E000C4F898101268C4F8942194F8C120C4F8D7
:10C1F00098210023D4F8C820C4F89C2184F8C130C9
:10C20000D4F8C420C4F8A021012384F8A83194F8FC
:10C21000B031092B06D194F89420022A04BF0522DC
:10C2200084F89420D4F8B421002A00F0D980092B96
:10C2300040F0D68094F89430012B40F0D180D4F8AF
:10C2400098101048002350F823508D4240F0C480CD
:10C25000052384F89430C3E00C80FF1F5896FF1F1D
:10C26000F495FF1FC093FF1F6B98FF1FA495FF1F3E
:10C270000896FF1F4487FF1F5C98FF1F7898FF1FD9
:10C280006096FF1F3088FF1F03A8FCF747FA05469A
:10C2900000284ED0FCF75AFA08B184F8E36194F80C
:10C2A000E3219DF80C10531CDBB22244092B84F8C7
:10C2B000E33182F8E4117FF41AAF604A94F8E41194
:10C2C00052780023914284F8E3317FF410AF5C4947
:10C2D0005A5C01331644082BF6B2F9D194F8EC31CC
:10C2E000B34222D1574B94F8E5211A7094F8E62115
:10C2F0005A7094F8E7219A7094F8E8219A7194F8AA
:10C30000E9215A7194F8EA211A7194F8EB21DA7054
:10C31000FCF7B2F94C4B4D4A18600023137003220E
:10C3200084F8B02184F8E3318EE6042384F8B03138
:10C33000DDE60AAE3046FCF740FC48B32B46F25C23
:10C3400001331544082BEDB2F9D19DF83020AA42F3
:10C35000ECD13C4B9DF829201A709DF82A205A7088
:10C360009DF82B209A709DF82C209A719DF82D2015
:10C370005A719DF82E201A719DF82F20DA70FCF763
:10C380007BF9314B1860314B00221A70072359E6B4
:10C3900094F89430013B012B3FF6A9AED4F89830C5
:10C3A000B3F5C05F0ED2FCF7C9FB58B1D4F89800C2
:10C3B0002449431CC4F89830FCF73BFD092384F85A
:10C3C000B03148E6002384F8943090E6D554013328
:10C3D0002F2B7FF4EDAE1AE701339A427FF433AF8F
:10C3E0000FB0BDE8F08394F8B001082804D840F2FB
:10C3F0005112C240D207F3D4D4F8AC01144DD3F893
:10C4000003306970B0F5C05F6B6012D20D49FCF764
:10C4100009FD0C49D4F8AC01FCF72FFD38B1D4F874
:10C42000AC310133C4F8AC3165232B70D8E7072356
:10C43000FBE707232B7000230BE700BF0C80FF1FD7
:10C440005C88FF1F5896FF1FFC95FF1F0696FF1F75
:10C450007098FF1F704710B5074CFCF70DF9236863
:10C46000C01AB0F5FA7F05D9044B0222DA60FCF756
:10C4700003F9206010BD00BF7C9CFF1F00F00F403F
:10C4800070477047704770477047704770477047F4
:10C49000014B53F8200070476888FF1F2DE9F74FC4
:10C4A000A94DEB69ABB1A94E347894B9FCF7E4F827
:10C4B000A74B1B68C01A0028EB69B8BF40429842DE
:10C4C00007D92046013401F01BFE062CF9D10123C7
:10C4D00033702B6AABB19F4E347894B9FCF7CCF82B
:10C4E0009D4B1B68C01A00282B6AB8BF4042984277
:10C4F00007D92046013401F003FE062CF9D10123AF
:10C500003370964CFCF7B8F894F8303004EB8303A2
:10C510009B69C01A0028B8BF40420A2830DDFCF7EA
:10C52000ABF8074694F83000202100F00103994051
:10C5300041F00101C9B2400801F0BCF894F8308024
:10C5400004EB880506466B6BC31A07EE903AAB699D
:10C55000FB1AB8EEE77A07EE903AF8EEE77AC7EE04
:10C56000276A16EE900A04F095F875A3D3E9002324
:10C5700004F0E4F804F07CFB44F82800AF616E633B
:10C5800094F83000202500F0010105FA01F141F096
:10C590001501C9B2400801F08DF810F040030746BC
:10C5A00000933DD094F8300000F0010105FA01F14C
:10C5B000C9B2400801F07EF80138C0B201280AD99A
:10C5C00094F8300000F0010105FA01F10122C9B22E
:10C5D000D04001F027F894F83000614B012600EAC2
:10C5E000060120251E5405FA01F15E4B41F00601BB
:10C5F0001E544FF6FF72C9B2F04001F013F894F8E0
:10C60000300000EA060105FA01F141F007010022BD
:10C61000C9B2F04001F006F894F83030524AD654CE
:10C6200094F83000514E06EB80131B69002B67D045
:10C6300000F00101202505FA01F141F00201C9B223
:10C64000400801F037F894F8303006EB83120028E8
:10C650001269B8BF4042904252D9E21892F84C2079
:10C66000BAB94FEA530903F001039D4045F01405A0
:10C67000EDB22946484601F01DF8294640F4806293
:10C68000484600F0CFFF94F830300122234483F86D
:10C690004C2094F85250DFF8E0B055B9E8B2FCF7FE
:10C6A000D2F90BF805000135082DF7D1012384F8E4
:10C6B00052302F49DFF8BCA027254FF000094FF07A
:10C6C00002085FFA89F00191FCF7BDF91BF8093007
:10C6D0000199834259D009F10C030BF8090051F874
:10C6E0002330022B4AD0032B03D0012B4DD100283D
:10C6F0004BD01AF80530012B08BF0AF8058044E03A
:10C7000094F83050631993F84C30002BC1D005F0E9
:10C7100001034FEA550920259D4045F01405EDB26F
:10C720002946484600F0C6FF294620F48062484664
:10C7300000F078FF94F8303000222344A7E700BFD0
:10C74000FCA9F1D24D6290400C80FF1F0696FF1F9E
:10C75000FC95FF1FC093FF1FF495FF1F6888FF1F04
:10C76000EA93FF1F5096FF1F0094FF1F0894FF1FBE
:10C77000A495FF1F0896FF1FBB88FF1F28B91AF852
:10C780000500012801D10AF8053009F10109B9F1C4
:10C79000080F05F1010594D194F8303017F001012C
:10C7A00004EB030200F0B88092F85B1091B901210C
:10C7B00082F85B10664A1A4492F8242012F0010FA6
:10C7C00008D002211B2211FB0323624AD05C0128FE
:10C7D00008BFD15494F83030E218B80792F86110CD
:10C7E00040F1A88091B9012182F86110584A1A4499
:10C7F00092F82A2012F0010F08D00E33554A12F891
:10C800001310012904BF022102F8131017F0800948
:10C8100008D094F830304F4A0333D15C012904BF6B
:10C820000221D154009B43B194F83030494A0F3370
:10C83000D15C012904BF0221D15494F8300006EBE9
:10C8400080131B6A9BB37D0531D400F001012025C4
:10C8500005FA01F141F01901C9B2400800F02AFFC0
:10C86000074694F8300000F0010105FA01F141F0AB
:10C870000101C9B2400800F01DFF94F8303006EB0A
:10C880008316381A0028326AB8BF404290420ED947
:10C89000184601F035FC94F830302F4A0121D1546C
:10C8A00015332C4AD15C012904BF0221D154B9F1BE
:10C8B000000F14D0294994F830300A7842FA03F076
:10C8C000C0070CD50120264D00FA03F32B70254D2F
:10C8D00028702548007810B922EA03030B7094F8F9
:10C8E0003000202100F00103994041F01501C022E1
:10C8F000C9B2400800F096FE94F8300000F074F8D9
:10C9000094F830300133DBB2052B88BF002384F864
:10C91000303003B0BDE8F08F92F85B0000283FF4A0
:10C9200059AF82F85B100A4A1A4492F8242012F098
:10C93000020F45E700293FF469AF012182F8611039
:10C94000034A1A4492F82A2012F0020F54E700BF5B
:10C95000A495FF1F0896FF1FE493FF1FF193FF1F8D
:10C96000F093FF1F5696FF1FDC93FF1F2DE9F34145
:10C970001A4C235C06460F4600F0010845086BB1CF
:10C980002021174B01FA08F141F0060153F820204D
:10C99000C9B2284600F046FE0023A355202404FA1D
:10C9A00008F4EDB244F0070187EAE772A2EBE77200
:10C9B0002846C9B200F036FE0A4B0122002F9A55D4
:10C9C0004FF00003D8BF02220192E1B200931A4651
:10C9D000284600F0CDFD02B0BDE8F0815096FF1F63
:10C9E0003896FF1FEA93FF1F2DE9F04F202287B0F2
:10C9F00000F0010302FA03F303939DF90C50BC4FBE
:10CA0000460845F015010446C9B2304600F052FE12
:10CA10000146A00107EB000C4A089CF80830DCF83E
:10CA20000490059113F0400F14BF385857F800A038
:10CA300001F0010E1DBF02F0010BC0F1000A5FFA08
:10CA40008EF202F0010214BFC9F100095FFA8EFBF9
:10CA50001F0603F03F080492204615D501F07AFB2B
:10CA6000049A0599B0FA80F35B0908F1FF300728B2
:10CA700000F2B981DFE810F0100010001000100083
:10CA8000460146014601460101F064FB031C18BF44
:10CA900001230599049AE8E7964F3B5D013B0E2B75
:10CAA00000F2A181DFE813F00F0021003200410005
:10CAB00053005C006D007C00B600E200E8009F01BE
:10CAC0001F013702320245F01401C9B2304600F0AE
:10CAD000F1FD07EB840301229860A8F10208864B60
:10CAE00090451A551ED802231DE007EB84039A686F
:10CAF00045F0140142F00202C9B2304600F092FD46
:10CB000051462046FFF732FF03230CE0002A00F0D5
:10CB10006A8145F00101C9B2304600F0CBFD774B88
:10CB200043F8240004233B555DE107EB84039A6836
:10CB300045F0140142F00102C9B2304600F072FD26
:10CB4000CAF100012046FFF711FF0523EBE7BBF117
:10CB5000000F00F04881204601F0D2FA0623E2E7F8
:10CB600007EB840345F014019A68C9B2304622F0FD
:10CB7000030200F057FD49462046FFF7F7FE072362
:10CB8000D1E7BBF1000F40F02E8159462046FFF758
:10CB9000EDFEC9F100012046FFF7E8FE0823C2E7D9
:10CBA000BBF1000F00F01F8145F00101C9B2304612
:10CBB00000F080FD002180462046FFF7D7FE4F4A57
:10CBC00052F82430A3EB080342F8243007EB840327
:10CBD00045F014019A68C9B222F00302304600F011
:10CBE00021FD45F007014A46C9B2304600F01AFD62
:10CBF00045F00D014246C9B2304600F013FD002356
:10CC0000019300931A469DF80C10304600F0B0FCDA
:10CC1000092388E7890540F1E68045F0010A5FFABB
:10CC20008AFA5146304600F045FD354B0021186028
:10CC30002046FFF79BFE45F00D010022C9B23046A9
:10CC400000F0F0FC00225146304600F0EBFC45F0CD
:10CC500019010022C9B23046A8F1030800F0E2FC35
:10CC6000B8F1010F41D8C9F10001D4E0BBF1000FC8
:10CC700000F0B9800B2356E7BBF1000F40F0B38002
:10CC800045F00101C9B2304600F014FD5946804616
:10CC90002046FFF76BFE07EB840345F014019A680A
:10CCA000C9B222F00302304600F0BCFC45F0070197
:10CCB0004A46C9B2304600F0B5FC45F00D010222EB
:10CCC000C9B298FBF2F2304600F0ACFCCDF804B0EB
:10CCD000CDF800B05B461A469DF80C10304600F0C7
:10CCE00047FC0D231FE78A057DD50E231BE700BFF8
:10CCF0000894FF1FD088FF1FEA93FF1FC493FF1FF4
:10CD00008C95FF1F894F385D01380E286BD8DFE8FE
:10CD100010F00F002400390047005C006A006D002D
:10CD20006A006A009D00A9008700D6000201FD008C
:10CD30007F4B45F014010122C9B230461A5500F06C
:10CD4000B9FC07EB8403B8F1060F98603FF4CBAE53
:10CD5000B8F1080F7FF4E6AEC5E6B8F1060F05D1CD
:10CD600007EB84039A6822F00302C1E6B8F1080FCA
:10CD70007FF4C6AE07EB840345F014019A6822F0F5
:10CD80000302B9E6A8F10501012906D82AB1B8F1D4
:10CD9000060F3FF4C7AE0F23C5E623B30C23C2E64C
:10CDA000B8F1050F05D107EB84039A6822F003025E
:10CDB000BEE6B8F1070F7FF4C3AE07EB840345F07E
:10CDC00014019A6822F00302B6E6A8F10502012ACE
:10CDD00006D8BBF1000F03D0B8F1050FDBD182E616
:10CDE000002B7FF4CCAE07B0BDE8F08F002BFAD15A
:10CDF000A8F10708B8F1010F0CD907EB840345F03F
:10CE000014019A6822F0030242F00202C9B23046CD
:10CE100000F008FC49462046FFF7A8FD0A2382E6F9
:10CE2000002BE0D1A8F10708B8F1010F7FF61BAF86
:10CE300007EB840345F014019A6822F0030242F0E4
:10CE40000102C9B2304600F0EDFB0CE7002BCAD05E
:10CE500045F00101C9B2304600F02CFC07EB840319
:10CE6000186207E7002BBED145F00101C9B207EBFC
:10CE7000840A3046049300F01DFCDAF8082045F0DF
:10CE80001401804622F00302C9B2304600F0CAFB0A
:10CE900045F007014A46C9B2304600F0C3FBDAF854
:10CEA000202045F00D019044C9B20222304698FB83
:10CEB000F2F200F0B7FB049B019300930BE78B05A4
:10CEC00091D50E233B5545F00107FFB23946304658
:10CED00000F0F0FB174B002118602046FFF746FDDD
:10CEE00045F00D0130460022C9B200F09BFB3946E7
:10CEF0003046002200F096FB45F019010022C9B22D
:10CF0000304607B0BDE8F04F00F08CBB0021204652
:10CF1000FFF72CFDE9E607EB840345F014019A685E
:10CF2000C9B2304600F07EFB0023FCE5D088FF1F2D
:10CF3000EA93FF1F8C95FF1F024B1A5C0AB901226E
:10CF40001A547047D088FF1F024B1A5C0AB10F2297
:10CF50001A547047D088FF1F014B185C704700BF00
:10CF6000D088FF1F0C4A116940F273234B434FF6E0
:10CF7000FF71B3FBF1F36E2B06D9084B4FF4802100
:10CF800059605723136070474F2B9EBF034B4FF4DC
:10CF900080219960F5E700BF00B0034080F00F40AA
:10CFA0001B4B1A6802F01F02072A2ED8DFE802F096
:10CFB000040B2D11171D23291A69164992B20A80F4
:10CFC00041221A6070471A69124992B24A8043227C
:10CFD000F7E71A690F4992B2CA804422F1E71A6949
:10CFE0000C4992B20A814522EBE71A69094992B2CB
:10CFF0004A814622E5E71A69064992B28A814722A8
:10D00000DFE71A69034992B2CA814022D9E700BF1B
:10D0100000B00B400889FF1F38B541F23001114BB9
:10D020005A5842F000625A5041F23C0100245A58CA
:10D0300042F000625A5003F5E8230C2540229D601F
:10D040004920DC605C621A6001F016FA064B572238
:10D050009D602720DC605C621A60BDE8384001F00A
:10D060000BBA00BF0070044000B003400B2829D861
:10D07000DFE800F0060A0D102828282813281E23B0
:10D08000114B188980B270470F4B5889FAE70E4B45
:10D090009889F7E70C4BD889F4E70B4B588883B293
:10D0A00040F2732058434FF6FF7390FBF3F0704744
:10D0B000054BD88883B28E20F4E7034B188883B2DF
:10D0C0004220EFE7002070470889FF1F30B52E4D42
:10D0D00041F23C042B5943F010032B512B4B4FF4DE
:10D0E00000741C636FF4F8755C63A3F51433A4F14A
:10D0F0003E542C441C604FF400545C60244C1C6073
:10D100001C68E401FCD50138072834D8DFE800F0BA
:10D11000312F2D2B293327041E4858601E4B002029
:10D1200058631E4818601E484FF0806400EA81452D
:10D13000C3F88040C3F88450FAB100EA8240C3F8D3
:10D140009040C3F894004FF08460C3F8A000C3F887
:10D15000A410AAB1C3F8B000C3F8B42030BD114880
:10D16000DBE71148D9E71148D7E71148D5E711485F
:10D17000D3E71148D1E71148CFE7C3F89020E2E7A1
:10D18000C3F8B02030BD00BF0070044000900440E0
:10D190000F0080508720FE01004002400F008000F9
:10D1A0000000FC1F8720FE038720FE0F8720FE1350
:10D1B0008720FE278720FE638720FEC78720FE0783
:10D1C000384AD2F88030C3F30363022B5FD0D2F821
:10D1D0009030C3F30363022B5BD0D2F8A030C3F3CB
:10D1E0000363022B06D0D2F8B030C3F30363022BE3
:10D1F00056D103231B0103F1402202F50032D2F87D
:10D200008010C1F303410170D2F8801011F4801135
:10D2100018BF01218170D2F8801011F4001118BFDD
:10D22000012141704178B1BBD2F88410C1F38A4129
:10D2300003F1402303F500334160D3F88810090E51
:10D240000172D3F88810090C4172D3F88810090ACA
:10D250008172D3F88810C172D3F88C10090E017353
:10D26000D3F88C10090C4173D3F88C10090A817320
:10D27000D3F88C30C373D2F880309B024CBF4FF090
:10D2800084634FF08063C2F8803001207047002330
:10D29000B0E70123AEE7D2F8841021F06041C7E780
:10D2A0000020704700400240184AD2F87031C3F3A2
:10D2B00003630C2B10B527D04478436804B3C3F341
:10D2C0001103C2F874318368104A1BBAC2F878316E
:10D2D000C3681BBAC2F87C318378002C14BF4FF0AE
:10D2E00042624FF040620BB142F4801203781B049B
:10D2F00003F470231343054A0120C2F8703110BDB6
:10D30000034901EA8343DCE7002010BD00400240EE
:10D310000000FC1F0B4B4FF00062C3F870214FF46C
:10D320008022C3F87421084AC3F878216FF484710D
:10D33000A2F166320A44C3F87C21044AC3F8702182
:10D34000704700BF00400240785634120000080CBD
:10D3500010B53A4BDA7842F00202DA70384A1078A7
:10D36000C0B20228114641D0032835D0012832D15D
:10D37000546891688C4215D2D978C90707D451688E
:10D38000D0684C1C5460425CD2B21A7110BD9978BE
:10D3900001F0DF019970997801F0EF019970107434
:10D3A000002317E0517C01F0FF0049B9997801F0A2
:10D3B000DF019970997801F0EF019970107010BD3C
:10D3C000997841F004019970917CC9B219710023D8
:10D3D00053740323137010BD997801F0EF01997015
:10D3E0001B795169DBB20B700223F3E79469D069B2
:10D3F00084421DD2D2698869121A012A05D19A780D
:10D4000002F0DF029A7000230B70CB698A699B1AC5
:10D41000022B9FBF094A937843F0080393708A69EF
:10D420004869531C8B61054B1B79DBB2835410BDDB
:10D43000997801F0DF019970B2E700BF00700640F3
:10D440001C89FF1F41F234020A498B5843F08003C4
:10D450008B50094B4FF418729A62DA6203F5E0338D
:10D460001B225A70C0229A7000225A71192001F0B2
:10D4700003B800BF0070044000B0044010B5104B6A
:10D4800000241C745C749A6001225C601A700D4A5E
:10D49000D960917801F0F7019170917841F0100115
:10D4A0009170917800F0FE0041F0200191701071B0
:10D4B0001A78002AFCD1187CB0FA80F0400910BD1F
:10D4C0001C89FF1F0070064010B5104B00241C740F
:10D4D0005C74DA6103229C611A700D4A596191787B
:10D4E00001F0F7019170917841F0100191709178FD
:10D4F00040F0010041F02001917010711A78002A6B
:10D50000FCD1187CB0FA80F0400910BD1C89FF1FC7
:10D510000070064070B5144C002563610126049B21
:10D5200025746674A2606560E36140EA0603A56144
:10D53000A3740E4BE16026709A7802F0F7029A709D
:10D540009A7842F010029A709A7800F0FE0042F049
:10D5500020029A7018712378002BFCD1207CB0FA3D
:10D5600080F0400970BD00BF1C89FF1F007006409D
:10D570002DE9F74F01F07F0493461502352C4FEA51
:10D580004402984682469DF830709DF83460234BE3
:10D59000019201D0552C17D148EA050547EA052725
:10D5A0006200224446EA0726924426F4736626F077
:10D5B0000306F60453F82A20F60C22EA060643F87E
:10D5C0002A6003B0BDE8F08F154A019332F810903D
:10D5D00041F0800100224846FBF75AFB00225946E1
:10D5E0004846FBF755FB002241464846FBF750FBF7
:10D5F000394600224846FBF74BFB3146012248469C
:10D60000FBF746FB48EA05056300234447EA052784
:10D610009A4446EA0726019BD1E700BF3C89FF1FD9
:10D62000D81201002DE9F84301F07F06352E81461E
:10D630001546DFF87C804FEA460401D0552E0FD105
:10D6400034444C4425F4736525F0030558F8243020
:10D65000ED04ED0C23EA050348F82430BDE8F88317
:10D66000124B33F81070002241F080013846FBF76E
:10D670000FFB0022290E3846FBF70AFB3444002238
:10D68000C5F307413846FBF703FB4C440022C5F3C2
:10D6900007213846FBF7FCFA0122E9B23846FBF7CE
:10D6A000F7FA48F82450BDE8F88300BFD81201000B
:10D6B0003C89FF1FF8B5334B01F07F055A19064628
:10D6C000127B002A56D033F81070002229463846C3
:10D6D000FBF7DEFA002211463846FBF7D9FA0022A2
:10D6E00011463846FBF7D4FA002211463846FBF7BC
:10D6F000CFFA012200213846FBF7CAFA0022114670
:10D700003846FBF7C5FA002211463846FBF7C0FA47
:10D710000022114604023846FBF7BAFA00221146ED
:10D7200004433846FBF7B4FA2402044301220021E3
:10D730003846FBF7ADFA2402352D40EA040001D04B
:10D74000552D0ED105EB45030F4A1E4452F82630E5
:10D7500023F4736323F00303DB04DB0C184342F868
:10D760002600222D01D0422D0AD1030208D540F017
:10D770007F40F8BD05EB45050544034B53F82500F4
:10D78000F8BD00BFD81201003C89FF1FF8B50E4D4F
:10D7900005440E4695F8003693B9040104F01004D0
:10D7A000470844F06C0421463846FFF783FF06F033
:10D7B0000F0320F00F021A4321463846FFF732FFCD
:10D7C00085F80666F8BD00BF3C89FF1F70B50401EF
:10D7D00004F01004460844F06C040D46304621461F
:10D7E000FFF768FF2D0105F0700520F070022A4355
:10D7F00021463046BDE87040FFF714BF70B5040104
:10D8000004F01004460844F06C040D4630462146EE
:10D81000FFF750FFED0305F4C03520F4C0322A4372
:10D8200021463046BDE87040FFF7FCBE70B50401EC
:10D8300004F01004460844F06C040D4630462146BE
:10D84000FFF738FF2D0505F4700520F470022A4318
:10D8500021463046BDE87040FFF7E4BE70B50401D4
:10D8600004F01004460844F06C040D46304621468E
:10D87000FFF720FF2D0605F0706520F070622A4347
:10D8800021463046BDE87040FFF7CCBE70B50401BC
:10D8900004F01004450844F06C040E462846214666
:10D8A000FFF708FF3EB140F0804221462846BDE820
:10D8B0007040FFF7B7BE20F08042F6E770B5040174
:10D8C00004F01004450844F06C040E462846214636
:10D8D000FFF7F0FE3EB140F4002221462846BDE8A5
:10D8E0007040FFF79FBE20F40022F6E770B50401F8
:10D8F00004F01004450844F06C040E462846214606
:10D90000FFF7D8FE3EB140F4802221462846BDE80C
:10D910007040FFF787BE20F48022F6E770B504015F
:10D9200004F01004450844F06C040E4628462146D5
:10D93000FFF7C0FE3EB140F4804221462846BDE8D4
:10D940007040FFF76FBE20F48042F6E770B5040127
:10D9500004F01004450844F06C040E4628462146A5
:10D96000FFF7A8FE3EB140F4005221462846BDE82C
:10D970007040FFF757BE20F40052F6E770B504017F
:10D9800004F01004450844F06C040E462846214675
:10D99000FFF790FE3EB140F4805221462846BDE894
:10D9A0007040FFF73FBE20F48052F6E770B50401E7
:10D9B00004F01004460844F06C040D46304621463D
:10D9C000FFF778FE2B0748BF20F070004FEA0512E2
:10D9D0004CBF40F4006020F4076002F07002024384
:10D9E00021463046BDE87040FFF71CBE70B504010B
:10D9F00004F01004460844F06C040D4630462146FD
:10DA0000FFF758FEED0105F4F06520F4F0622A43BB
:10DA100021463046BDE87040FFF704BEFFF7E6BF81
:10DA200070B5040104F01004450844F06C040E467F
:10DA300028462146FFF73EFE3EB140F40032214623
:10DA40002846BDE87040FFF7EDBD20F40032F6E750
:10DA500008B5094B034493F8002652B9010101F0BF
:10DA6000100141F06C014008FFF724FE00F00F00A8
:10DA700008BD93F8060608BD3C89FF1F010108B5E3
:10DA800001F0100141F06C014008FFF713FEC0F3F4
:10DA9000021008BD010108B501F0100141F06C0150
:10DAA0004008FFF707FEC0F3C13008BD010108B50B
:10DAB00001F0100141F06C014008FFF7FBFDC0F3DD
:10DAC000035008BD010108B501F0100141F06C01DF
:10DAD0004008FFF7EFFDC0F3036008BD010108B582
:10DAE00001F0100141F06C014008FFF7E3FDC0F3C5
:10DAF000807008BD010108B501F0100141F06C0112
:10DB00004008FFF7D7FDC0F3C04008BD010108B5CC
:10DB100001F0100141F06C014008FFF7CBFDC0F3AC
:10DB2000804008BD010108B501F0100141F06C0111
:10DB30004008FFF7BFFDC0F3803008BD010108B504
:10DB400001F0100141F06C014008FFF7B3FDC0F394
:10DB5000403008BD010108B501F0100141F06C0131
:10DB60004008FFF7A7FDC0F3003008BD010101F038
:10DB7000100108B541F06C014008FFF79BFDC0F3B0
:10DB80000213020548BF43F00803184608BD01010F
:10DB900008B501F0100141F06C014008FFF78AFD63
:10DBA000C0F3C31008BDFFF7F2BF010108B501F0D3
:10DBB000100141F06C014008FFF77CFDC0F34040CC
:10DBC00008BD70B5040104F01004460844F06D046B
:10DBD0000D4630462146FFF76DFD6D0105F06005ED
:10DBE00020F060022A4321463046BDE87040FFF72E
:10DBF00019BD70B5040104F01004460844F06D042A
:10DC00000D4630462146FFF755FD6D0305F4C0452E
:10DC100020F4C0422A4321463046BDE87040FFF759
:10DC200001BD70B5040104F01004460844F06D0411
:10DC30000D4630462146FFF73DFD2D0205F4706587
:10DC400020F470622A4321463046BDE87040FFF759
:10DC5000E9BC70B5040104F01004460844F06D04FA
:10DC60000D4630462146FFF725FD05F00F0520F053
:10DC70000F022A4321463046BDE87040FFF7D2BC70
:10DC800070B5040104F01004450844F06D040E461C
:10DC900028462146FFF70EFD20F47F0040EA0642A9
:10DCA00021462846BDE87040FFF7BCBC70B50401B2
:10DCB00004F01004450844F06D040E462846214641
:10DCC000FFF7F8FC3EB140F4004221462846BDE88B
:10DCD0007040FFF7A7BC20F40042F6E770B50401DE
:10DCE00004F01004450844F06D040E462846214611
:10DCF000FFF7E0FC3EB140F0807221462846BDE8C7
:10DD00007040FFF78FBC20F08072F6E7010108B584
:10DD100001F0100141F06D014008FFF7CBFCC0F3AA
:10DD2000411008BD010108B501F0100141F06D017D
:10DD30004008FFF7BFFCC0F3413008BD010108B542
:10DD400001F0100141F06D014008FFF7B3FCC0F392
:10DD5000032008BD010108B501F0100141F06D017B
:10DD60004008FFF7A7FC00F00F0008BD010101F01B
:10DD7000100108B541F06D014008FFF79BFC03144A
:10DD8000D8B21B0648BF60F0FF0008BD010108B50E
:10DD900001F0100141F06D014008FFF78BFCC0F36A
:10DDA000C03008BD010108B501F0100141F06D015E
:10DDB0004008FFF77FFCC0F3006008BD10F0010FC2
:10DDC00070B514BF1826102645080C462846314663
:10DDD000FFF770FC04F0030420F4401242EA0452FE
:10DDE00031462846BDE87040FFF71CBC10F0010F1B
:10DDF00070B514BF1825102544080E462046294644
:10DE0000FFF758FC3EB140F4802229462046BDE889
:10DE10007040FFF707BC20F48022F6E710F0010FF6
:10DE200070B514BF1826102645080C462846314602
:10DE3000FFF740FC04F0030420F4403242EA0442BD
:10DE400031462846BDE87040FFF7ECBB10F0010FEB
:10DE500070B514BF1825102544080E4620462946E3
:10DE6000FFF728FC20F47F4040EA0622294620469E
:10DE7000BDE87040FFF7D6BB10F0010F70B514BFBE
:10DE80001825102544080E4620462946FFF712FCA7
:10DE900020F0FF0046EA000229462046BDE8704017
:10DEA000FFF7C0BB10F0010F08B514BF18211021F7
:10DEB0004008FFF7FFFBC0F3015008BD10F0010F51
:10DEC00008B514BF182110214008FFF7F3FBC0F379
:10DED000804008BD10F0010F08B514BF18211021B3
:10DEE0004008FFF7E7FBC0F3014008BD10F0010F49
:10DEF00008B514BF182110214008FFF7DBFBC0F361
:10DF0000072008BD10F0010F08B514BF182110211B
:10DF10004008FFF7CFFBC0B208BD10F0010F08B5F5
:10DF200014BF192111214008FFF7C4FBC0B208BD7E
:10DF30002DE9F743FAF7A0FB0446FAF79DFB001B17
:10DF40000028B8BF40420928F7DD0026B046F4B2E9
:10DF500001254FF035092B4600226C21204614275D
:10DF60008DE82002FFF704FB072300223021204622
:10DF7000CDF804800097FFF7FBFA2B4600227C21A6
:10DF800020468DE82002FFF7F3FA072300225021F4
:10DF900020468DE88001FFF7EBFA0022114620466B
:10DFA000FFF740FB002220212046FFF73BFB002229
:10DFB0002D212046FFF736FB002221212046FFF7C6
:10DFC00031FB002240212046FFF72CFB00224D218F
:10DFD0002046FFF727FB002241212046FFF722FBC6
:10DFE0002A4623212046FFF71DFBDC222421204660
:10DFF000FFF718FB46F6DB0225212046FFF712FB50
:10E0000040F2B71226212046FFF70CFB4DF2B71263
:10E0100027212046FFF706FB40F2B71228212046B1
:10E02000FFF700FBDC222A212046FFF7FBFA0A2239
:10E030002B212046FFF7F6FA2A4643212046FFF718
:10E04000F1FADC2244212046FFF7ECFA46F6DB0227
:10E0500045212046FFF7E6FA40F2B7124621204656
:10E06000FFF7E0FA4DF2B71247212046FFF7DAFA40
:10E0700040F2B71248212046FFF7D4FADC224A21A9
:10E080002046FFF7CFFA2E440A224B212046FFF705
:10E09000C9FA032E7FF45BAF074D0024AE1F27465D
:10E0A000E0B2FFF7D5FCA75528550134062CF7D16F
:10E0B00003B0BDE8F08300BF428FFF1F38B5074CA7
:10E0C000044494F8001641B994F80656FFF75EFB35
:10E0D000012384F8003684F8065638BD3C89FF1FBA
:10E0E000064B034493F8002632B1002293F806163B
:10E0F00083F80026FFF74ABB704700BF3C89FF1F2B
:10E10000124BF7B501271F54114BC0F347061F549C
:10E1100020243840844065B245F007013046002293
:10E12000C9B2FFF77FFA45F0060130464FF6FF729D
:10E13000C9B2FFF777FA0023019700931A46E1B2BC
:10E140003046FFF715FA03B0F0BD00BFEA93FF1F9A
:10E150005096FF1F10F0010F08B54FF004014FEA71
:10E16000500004D0FFF7A6FAC0F3401008BDFFF737
:10E17000A1FAC0F3001008BD002808B50FDB02F0BB
:10E1800077FA0DA3D3E9002302F002FC41EC100B57
:10E1900002F0DAFF51EC100B02F06AFD08BD02F04C
:10E1A00067FA05A3D3E9002302F0F2FB41EC100B60
:10E1B00002F036FFEEE700BF34F7FFFF7F84EE3F4B
:10E1C00008B502F055FA08A3D3E9002302F0E0FBFA
:10E1D00041EC100B02F0B8FF51EC100B02F048FDBF
:10E1E00008BD00BFAFF30080EB1100A2941A5D40A0
:10E1F000002808B50FDB02F03BFA0DA3D3E900239A
:10E2000002F09CFA41EC100B02F00AFF51EC100BEB
:10E2100002F02EFD08BD02F02BFA05A3D3E900237E
:10E2200002F08CFA41EC100B02F08EFFEEE700BF1B
:10E2300034F7FFFF7F84EE3F08B502F019FA08A318
:10E24000D3E9002302F07AFA41EC100B02F0E8FE69
:10E2500051EC100B02F00CFD08BD00BFAFF30080C5
:10E26000EB1100A2941A5D40704700BF000000004F
:10E2700038B500242025E0B200F0010105FA01F1D3
:10E2800041F01A014FF48032C9B240080134FFF75F
:10E29000C9F9062CEFD138BD2DE9F74F5A4E06EBE0
:10E2A00080164408F36900F0010723B1B6F81A801C
:10E2B000B8F1000F1BD12025BD406DB245F0180606
:10E2C000E4B2F6B231462046FFF7F4F9314620F4C5
:10E2D00080622046FFF7A6F945F01A014FF480321C
:10E2E000C9B2204603B0BDE8F04FFFF79BB9FFF776
:10E2F000E9FBC0F1080008FA00F002F0B9F9F5698D
:10E30000804685EAE570A0EBE570894602F0B0F939
:10E3100002460B464046494602F03AFB00223B4B80
:10E3200082468B4602F00AFA8946804649EC108BF9
:10E33000684602F08DFD0022002351EC100B02F024
:10E3400065FCF8B14046494602F092FC002D4FF0C2
:10E35000200505FA07F56DB245F01806E4B2F6B2ED
:10E3600080463146B8BFC0F100082046FFF7A2F949
:10E37000314620F480622046FFF754F945F01A0137
:10E380004246ADE768464BEC10AB02F061FD002D54
:10E3900059EC108BDDE9000121DD02F069FC18A3C6
:10E3A000D3E9002306044946404602F0C7F902F0CB
:10E3B0005FFC2025BD406DB245F01807E4B2FFB206
:10E3C000064339462046FFF775F9394640F4806226
:10E3D0002046FFF727F945F01A01324680E702F0A0
:10E3E00047FCC04306A3D3E9002306044946404640
:10E3F00002F0A4F902F03CFCC0F51C501030D8E744
:10E40000000000000088C3400894FF1F0000F04097
:10E4100000F001032021994041F01901C9B24008E0
:10E42000FFF748B900F001022023934043F019039D
:10E430000A464008D9B2FFF7F5B800BFFEE74FF033
:10E44000E0210B4A0B4BC1F8083D4CF22053D3811D
:10E450004DF62813D381138823F001031B041B0CF2
:10E460001380D1F8883D43F47003C1F8883D7047AC
:10E470000020054000800000802800F01F014FF0C0
:10E4800001030F4A04DD8B40C2F88C31D360704722
:10E49000402804DD8B40C2F8883193607047202803
:10E4A00004DD8B40C2F8843153607047404200F075
:10E4B0001F0058BF41428B40C2F880311360704743
:10E4C00000E100E0802800F01F024FF001030D4939
:10E4D00003DD9340C1F88C307047402803DD934042
:10E4E000C1F888307047202803DD9340C1F884309C
:10E4F0007047404200F01F0058BF42429340C1F8AD
:10E500008030704700E100E0074B1A78D2B2012A50
:10E5100002D1222903D15A7001225A707047212951
:10E52000FAD10022F7E700BF488FFF1F70B51546EC
:10E5300011B91B4B197070BD022903D1184B012270
:10E540001A7070BD04291AD1154B5B78012B25D1A7
:10E550009488402C28BF402400235E1CDBB2A342D9
:10E5600007D300231A4602211846BDE8704000F088
:10E5700047BF2A68D05C00F0C3F83346EDE70329B3
:10E5800006D1074A5378012B08D100239370E9E79D
:10E59000052901BF024B00221A705A7070BD00BFDE
:10E5A000488FFF1F10B50446204600F0C1F8002830
:10E5B000FAD110BD704738B50A4C012502460B460A
:10E5C00000202946A57000F0F5FA224618B1002374
:10E5D000A370122038BD937803F0FF00002BFAD10E
:10E5E00038BD00BF488FFF1FF8B506460F4600F044
:10E5F000F4FC0E4B1A78012A16D15B78012B13D14B
:10E6000000F000F988B10025ECB2A74205D82146F8
:10E610003046BDE8F840FFF7CEBF301900F0D6F81D
:10E6200001350028F0D0F2E70C20F8BD488FFF1F1D
:10E6300008B540210248FFF7D7FF00F095F808BD64
:10E640004B8FFF1F38B5054600F0A8F80B2804468D
:10E6500009D140210548FFF7C7FF28B92846BDE882
:10E66000384000F09BB80024204638BD8B8FFF1F38
:10E6700070B50C46461E00250CB9284670BD16F82C
:10E68000010FFFF7DFFF013C002818BF0B25A4B2E4
:10E69000F2E738B5451E002415F8010F08B92046E9
:10E6A00038BDFFF7CFFF002818BF0B24F4E707B5EC
:10E6B0000123002200930649064B104600F020FA81
:10E6C000002814BF1B20002003B05DF804FB00BF2E
:10E6D0002DE5000009E5000038B50C46054600F0C0
:10E6E00097F8A0420AD32C440020A54207D000B1DD
:10E6F00038BD15F8010B00F051F8F6E70B2038BDD6
:10E7000010B50A4A117840290ED05378D418013335
:10E71000DBB2402BA07001F101014FF0000011703D
:10E7200014BF5370507010BD0B2010BDCB8FFF1F56
:10E7300010B50C4A117891B192F84230D4180133D7
:10E74000DBB2A4780470402B4FF0000001F1FF31E0
:10E75000117014BF82F8423082F8420010BD0A20C6
:10E7600010BD00BFCB8FFF1F014B1878704700BF53
:10E77000CB8FFF1F024B1878C0F14000C0B270472A
:10E78000CB8FFF1F034B00225A7083F842201A7070
:10E79000704700BFCB8FFF1FFFF7F4BF10B50A4AC9
:10E7A000117840290ED05378D4180133DBB2402BB6
:10E7B000A07001F101014FF00000117014BF5370FF
:10E7C000507010BD0B2010BD0E90FF1F10B50C4AED
:10E7D000117891B192F84230D4180133DBB2A478A9
:10E7E0000470402B4FF0000001F1FF31117014BF95
:10E7F00082F8423082F8420010BD0A2010BD00BFEE
:10E800000E90FF1F014B1878704700BF0E90FF1F3E
:10E81000024B1878C0F14000C0B270470E90FF1F45
:10E82000034B00225A7083F842201A70704700BFD1
:10E830000E90FF1FFFF7F4BF70B50546007801F09A
:10E8400093F902780023D9B2914207D25C1C03EB02
:10E85000830303445E786B789E4227D1174C2B7A52
:10E86000342202FB0142D67813B334234B43E2181F
:10E87000907886420CD000F0030204330C2010FB89
:10E8800002302118205C0B894A68497800F090FB1F
:10E89000D4F89C3083B12A46287812F8081F002942
:10E8A0000CBF03210521BDE8704018472346CAE785
:10E8B000937801339370D8E770BD00BF5490FF1F69
:10E8C0002DE9F04F85B00D4690468DF80F0001F010
:10E8D0004BF9022D064647D1077800235C1CDBB2BA
:10E8E000BB4210DB4FF00009DFF8B0B0CA465FFA58
:10E8F00089F4A74212DC284BD3F89C30002B45D179
:10E9000005B0BDE8F08F03EB830333440DF10F0036
:10E91000DA78597801F0E2F92346DFE704EB840462
:10E920003444E378A2886178CDF804A0A078009000
:10E930000DF10F0001F0B0F9A378032B05D15A4671
:10E9400061789DF80F0001F031FA6178E37841F0C9
:10E95000100141EAC3110022C9B20DF10F0001F00C
:10E96000EDF909F10109C2E7002DC4D10A49037884
:10E97000342000FB03138A1C3633294634329A4272
:10E98000B9D002F8341C02F8331CF7E74246294696
:10E990009DF80F009847B3E75490FF1F39E8000037
:10E9A000F0B40C7804F06004202C1D4632D14C7871
:10E9B000042C1DD00AD8012C04D003D3022C20D063
:10E9C000032C12D000202880F0BC7047212C1BD0D3
:10E9D00004D8202CF6D1F0BC00F040B9222C16D07F
:10E9E000232CEFD1F0BC00F049B9F0BC00F049B9DC
:10E9F00002241C801468002525701468671C1760A9
:10EA00006570F0BC00F056B9F0BC00F01FB9F0BC66
:10EA100000F076B9402C06D1044CD4F8A04014B1D3
:10EA2000A446F0BC6047CD20CEE700BF5490FF1F46
:10EA300073B50446007801F097F863680093A27AF2
:10EA4000637A43EA0223ADF8043002780023D9B296
:10EA5000914207D25D1C03EB830303445E78637825
:10EA60009E4225D1174D237A342202FB0152D678DB
:10EA700003B334234B43EA18907886420CD000F05D
:10EA8000030204330C2010FB02302918285C0B8988
:10EA90004A68497800F08CFAD5F89C3033B1227A74
:10EAA00020785AB104F108020521984702B070BDE0
:10EAB0002B46CCE7937801339370DAE76A4603215B
:10EAC000F3E700BF5490FF1F07B543680093437AF4
:10EAD000817A43EA0123ADF80430084BD3F89C3027
:10EAE00002462BB1017A007829B1083205219847F6
:10EAF00003B05DF804FB6A460421F8E75490FF1F59
:10EB00002DE9F84305460F461646984601F02CF8C5
:10EB100002789DF8203001328146D2B20021284689
:10EB200001F09EF80446E8B9164A1749284600F055
:10EB300086F999F80000154B342200FB022209F1F6
:10EB400001011A4499463433934201F105010CD175
:10EB50004146284600F074F8044618B9C9F89C707C
:10EB6000C9F8A0602046BDE8F88311F8050C03F849
:10EB7000340C11F8040C03F8330C03F8324C03F88E
:10EB8000314CE0E7A1E90000C1E800005490FF1F0C
:10EB900008B5074B0022C3F89C20C3F8A02000F062
:10EBA000A1F918B9BDE8084001F06EB808BD00BF72
:10EBB0005490FF1F2DE9F041984605460E46174632
:10EBC00000F0D2FF04780023D9B2A14207D201336A
:10EBD00003EB8302024412F8042CB242F4D1174C26
:10EBE00034234B43E218D07892F802E0A0EB0E01F8
:10EBF000C9B2042902D1C120BDE8F08100F00301AF
:10EC00000130C0B24FF00C0C0CFB0133D070A0EB04
:10EC10000E001C44C0B2012825716671A760A4F8DB
:10EC20000C8007D143463A4631462846BDE8F041BC
:10EC300000F0BEB90020BDE8F08100BF5490FF1F76
:10EC4000014B002019607047F890FF1F024B0979B3
:10EC5000197100F08DBF00BFF890FF1F13B500249D
:10EC600002AA1C80044B42F8041D0979197100F0B6
:10EC70008DFF02B010BD00BFF890FF1F002018806C
:10EC8000704730B40C460221198021796488084D00
:10EC9000012C297102D130BC00F08EBF022C02D1B0
:10ECA00030BC00F095BF0020188030BC704700BF1A
:10ECB000F890FF1F30B40C46022119802179648836
:10ECC000074D012C297102D130BC00F08DBF022C00
:10ECD00002D130BC00F09ABF0020188030BC7047D1
:10ECE000F890FF1F044B054A19795B791171137273
:10ECF00003210A23FFF75EBFF890FF1F4C80FF1F20
:10ED0000F8B500271F808B780B4CA371C3F3400329
:10ED10005A0063F3000206466271FFF7E3FF2568BD
:10ED200045B1A37913F002021ABF3A4622212121EC
:10ED30003046A8470020F8BDF890FF1F034B00F1B4
:10ED400008021B6800780521184700BF0091FF1FCB
:10ED500070B5094D04462A1D012100F0D7FF80221D
:10ED60000121204600F0EAFF2B68207800220A21CA
:10ED7000BDE87040184700BF0091FF1F37B5012163
:10ED80000DF10702044600F0C1FF9DF80730074D62
:10ED9000802B04D12A790121204600F0CFFF2B6877
:10EDA000207800220B21984703B030BD0091FF1F4F
:10EDB000436805215A7800F0C1BF73B501220024D1
:10EDC00005460126002100F089FF334621468DE8E3
:10EDD00050001022284600F05FFF224621462846B8
:10EDE00000F07CFF234621468DE850001022284683
:10EDF00000F052FF31460222284600F09FFF3246C3
:10EE00000621284600F09AFF22469021284600F06D
:10EE100095FF044B28781B682246214602B0BDE8C6
:10EE2000704018470091FF1F42783AB9C178C90174
:10EE300041F0100101F0900100F080BF704773B500
:10EE40000C468DF8070001F00DFA1F4D2C600446AA
:10EE5000002836D11D4A9DF80700102100F0A6FFBA
:10EE60001B4A044612219DF8070000F09FFF194A33
:10EE7000044314219DF8070000F098FFE4B2044316
:10EE8000154A9DF80700132100F090FFE4B20443F7
:10EE9000124A9DF80700172100F088FF02AEE4B285
:10EEA00004430F4A16F8010D162100F07FFFE4B26B
:10EEB000044303220121304600F040FF0323E4B263
:10EEC0002B71204602B070BD0091FF1FBBED00000A
:10EED000B1ED000051ED00007DED000029EE0000D5
:10EEE0003DED000037B502AD174B05F8010D0022CE
:10EEF000102128461A6000F05BFF122104462846C4
:10EF000000F056FF14210443284600F051FFE4B2FC
:10EF100004431321284600F04BFFE4B204431721B9
:10EF2000284600F045FFE4B204431621284600F0CD
:10EF30003FFFE4B2204310F0FF0003D19DF807002B
:10EF400001F09CF903B030BD0091FF1F1FB50121F6
:10EF50008DF807000DF10E020DF1070000F0D6FE4E
:10EF60000DF10F0206210DF1070000F0CFFE9DF814
:10EF70000E30802B18D19DF80F309B0714D59DF8CB
:10EF8000070000F0EFFD012804460DD172B60DF127
:10EF9000070000F029FB002221460DF107008DF843
:10EFA0000E2000F0CBFE62B69DF80E0004B010BD3E
:10EFB00073B50C4615461E468DF80700FFF7C6FFD1
:10EFC000802808D033462A4621460DF1070000F07C
:10EFD000A7FA02B070BD0020FBE77047062812D8E0
:10EFE00080000129C0B201D10230C0B2074AC0F38B
:10EFF0004703122101FB03231A884FF6FF739A423D
:10F0000008BFFF207047FF20704700BF0891FF1F17
:10F010002DE9F041314C324D324E4FF0000884F86A
:10F0200000814FF4107285F840020F462846FF21F8
:10F0300001F0C0FE4FF4806241463046C5F844629C
:10F0400001F0B8FE94F80C3143F0800384F80C31E1
:10F0500094F80C311B06FBD4234BFF221A7094F852
:10F060000C3143F0400384F80C31204B196897B3FE
:10F0700041F000411960194B310AC6F3074201F013
:10F08000FE0183F89C1083F8B020320E83F8B42080
:10F09000174AC5F84822102283F80821012283F874
:10F0A0009420BF2283F8802093F8002102F07F0291
:10F0B00083F8002193F8842042F0010283F8842031
:10F0C00093F8842042F0100283F8842084221A7777
:10F0D0000020BDE8F08121F00041CBE7002007408F
:10F0E0000891FF1F009EFF1F5680FF1F0070044005
:10F0F00000A0FF1F0D4B93F80C2102F0BF0283F814
:10F100000C21BF2283F8802093F8842002F0FE02B5
:10F1100083F8842093F8942002F0FE0283F8942070
:10F120001A7F02F07B021A77002070470020074008
:10F13000F7B5082304248DE81800B1F803300D78E2
:10F140008878B3F5007F81BF0023CB7002230B7159
:10F15000062D71D8AB00DCB2012804BF0234E4B242
:10F160004FEA540E354C122707FB0E474FF6FF7639
:10F17000B7F800C0B4455FD14E78032E5CD80128A3
:10F180005AD897F80FC0BCF1FF0F04BF4FF0000C26
:10F1900087F80FC0B1F803C0122101FB0EFE04EB8B
:10F1A0000E0743EA4003BA73FA7B7E7402F0010251
:10F1B00013435BB2D4F84822C7F80220D9B2F973DE
:10F1C0003874D4F8447224F80EC01BB207EBC30E97
:10F1D00081F00101CEF80420AEF802C04FF0080E15
:10F1E00007F833E007EBC10ECEF80420AEF802C0FA
:10F1F00012FA8CF24FF0480E07F831E0C4F84822BA
:10F2000028B917F8332062F07F0207F8332002AAEA
:10F2100002EB80002DB20A4950F8082C11F8253075
:10F22000012E0CBF164642F001063343DBB201F853
:10F230002530002003B0F0BD9520FBE70891FF1FAB
:10F24000C0200740084610B51146FFF7C7FEFF284B
:10F250001DD0104B1221C0F3470001FB0030D3F842
:10F260004422C37B1CB283F0010312F8341001F076
:10F270007F0102F8341012F8331001F07F0102F818
:10F2800033104FF0FF338372C372002010BDC420CF
:10F2900010BD00BF0891FF1F73B50C468DF8070025
:10F2A000114620461646FFF799FEFF28054620D056
:10F2B000214632460DF10700FFF7C4FFC5F34703AF
:10F2C00012210D4D59436B18D5F848221888121A8F
:10F2D000C5F8482224B2094A002002F824004FF061
:10F2E000FF326A549A705A70DA701A715A7102B009
:10F2F00070BD9620FBE700BF0891FF1FC0200740AC
:10F300002DE9F0410E468046114630461746FFF77C
:10F3100065FE0C4DC0F34700122303FB0050C47B75
:10F32000FF2C0DD03A4631464046FFF78BFF24B202
:10F33000D5F8442212F8343063F07B0302F83430FD
:10F34000BDE8F0810891FF1F10B508460021144662
:10F35000FFF744FE084AC0F34700122101FB0020DA
:10F36000D2F84432C27B03EBC2035A6813682360AD
:10F370005368636010BD00BF0891FF1F10B50C46B5
:10F3800020461146FFF72AFEFF281AD024B2104B60
:10F3900013F82430DBB213F00C0F12D09B0712D4F9
:10F3A0000C4BD3F8443213F83020D2090DD180F041
:10F3B0000100C0B213F83030DB0914BF0320002075
:10F3C00010BD052010BD012010BD032010BD00BFE1
:10F3D000C02007400891FF1F08B5FFF7FFFD074A4F
:10F3E0001223C0F3470003FB0020C37BFF2B1EBF8B
:10F3F000D2F84422002102F8331008BD0891FF1F03
:10F400002DE9F0410846002190461F46FFF7E6FD32
:10F410002249C0F34700122404FB0014E57BFF2DB2
:10F4200039D022884FF6FF7093B2834233D0D1F89F
:10F43000441285F0010011F9300000282BDB2EB2B8
:10F4400087B901EBC60338465A80D4F802205A60C7
:10F4500011F8352002F0400262F0770201F8362000
:10F46000BDE8F08101EBC602BB424FF0000028BFAF
:10F470003B466781C4F80680207360735380C2F8EE
:10F48000048011F8353003F0400363F0770301F88E
:10F490003630BDE8F0819420BDE8F0810891FF1F6F
:10F4A0002DE9F0410C460646114620461546FFF769
:10F4B00095FD194BC0F34700122202FB003090F873
:10F4C0000FE0BEF1FF0F24D027B2144A6CB1407C8C
:10F4D000012D0CBF14211821012818BF41F0010192
:10F4E00012F82700014302F8271012F827106FF3D3
:10F4F000410102F82710D3F84432002203F83E20DD
:10F500003DB92B462A4621463046BDE8F041FFF77B
:10F5100077BFBDE8F08100BF0891FF1FC020074002
:10F520002DE9F0410C462046012117469846FFF789
:10F5300055FDFF2836D01C4BC0F34700122202FBBA
:10F540000030D3F8446290F80FE016F93E30002BFB
:10F5500028DB23B2154A12F8235015F0020521D1F9
:10F560000188C0F806701FFA88F242818A42D8BF2B
:10F5700011460FFA8EF206EBC203057345735980EC
:10F580005F602CB9C82306F832302046BDE8F08110
:10F5900016F83E3003F0400363F0770306F832308C
:10F5A0002C46F2E79324F0E70891FF1FC0200740A4
:10F5B000034B044883F898100122114600F0BEBBAB
:10F5C000002007404893FF1F054B0648002283F8A0
:10F5D0009420802283F80C210121FF2200F0AEBB91
:10F5E000002007404893FF1F38B51A4C94F80021BB
:10F5F00002F07F0284F8002194F80C2102F0DF026F
:10F6000084F80C2194F8802042F0200284F88020B5
:10F6100094F8842002F0DF0284F8842094F8942087
:10F6200002F0DF0284F8942094F8942042F004025F
:10F6300084F8942044F62065013DADB200F0BCFE94
:10F64000002DF9D194F8943003F0FB0384F8943042
:10F6500038BD00BF002007402DE9F04FD84DD94CF0
:10F6600095F8807095F8843095F8906087B0FF2207
:10F670001F4094F840328DF809208DF80C308DF839
:10F680000D20002301210DF1090204F510708DF801
:10F690000E3004938DF815308DF816308DF80F303C
:10F6A0008DF8143000F032FB95F80C31D907F6B222
:10F6B0000FD59DF80930802B0BD195F8003103F060
:10F6C0007F0385F8003195F80C3103F0DF0385F8EE
:10F6D0000C317A0711D5BA4B042093F8A41093F893
:10F6E000A02083F8800006AB42EA012223F80E2D09
:10F6F00003A91220049300F06DFBFB074BD5B04D1E
:10F70000B0480123BF2685F8803085F8886095F8D9
:10F710009430002743F0020385F894304FF41072C0
:10F7200085F89870FF2185F8007101F043FB4FF4D4
:10F7300080623946D4F8440201F03CFBD4F84432EC
:10F7400003F50073C4F848329F4BFF221A7095F8F6
:10F75000943003F0FD0385F8943095F80C3143F0B4
:10F76000400385F80C319F2385F88C6085F8843040
:10F7700095F8943003F0DF0385F8943003A9102046
:10F7800000F028FB95F8943003F0DF0385F89430FF
:10F7900007B0BDE8F08F3D0740F19380884B082209
:10F7A00083F880203309C6F3C000062B8DF80D3096
:10F7B0008DF80F0000F2F480C6F3800202EB8302A2
:10F7C00008B10232D2B2D4F8446206EBC201C2F3ED
:10F7D0004705D1F804E04988ADF81510122101FB66
:10F7E0000541CDF810E091F80FC08CF0010C81F8C4
:10F7F0000FC016F8321082F0010A5FFA8AFAC1F3DC
:10F8000080110FFA8AF881F00101890106EBC8091D
:10F8100006F83810002800F0D980DFF8ACB19BB9A9
:10F820009BF8002082B9FF2219468BF8002003A81C
:10F830001A460193FFF706FD019B06F838301A4679
:10F84000194603A8FFF7DCFD9BF80030012B04D01C
:10F850009DF80D30002B00F0AD80122101FB054119
:10F86000BDF815008B894A8903449BB293428B8172
:10F8700009D3B1F800E0C0B2864540F09380897B9F
:10F88000012940F08F80122101FB0544D4F80610B5
:10F8900020881944D31A8342D8BF98B2A9F802002D
:10F8A000C9F8041016F83A3003F0400363F0770308
:10F8B00006F83830424A92F8943003F0DF0382F8B9
:10F8C0009430B80717D53E4C022384F8803094F862
:10F8D000883094F88C2003A9134016208DF814303A
:10F8E00000F078FABF2384F8883094F8943003F05D
:10F8F000DF0384F89430F9061CD5314C202384F8BA
:10F900008030102384F8803003A9142000F062FABC
:10F9100094F80C3143F0200384F80C3194F8003152
:10F9200043F0800384F8003194F8843043F02003DE
:10F9300084F88430BA060DD5214C202384F8803019
:10F9400003A9132000F046FA94F8843003F0DF0393
:10F9500084F884303B067FF51BAF0DF10A02FF23CC
:10F96000102103A88DF80D3000F0D0F99DF80A3071
:10F97000134C012B04BF8DF80F3000224FF0800391
:10F9800008BF8DF80D2003A984F88030172000F0FF
:10F9900021FA94F8943003F0DF0384F89430F7E60A
:10F9A000FF2210E7122202FB0544D4F8062004923D
:10F9B000ADF8153003A99DF80D0000F00BFA79E7BA
:10F9C000002007400891FF1F5680FF1F6BB916F8F3
:10F9D00032202F4902F03C02342A35D101238DF820
:10F9E0000E309EF80030DB090B70122101FB05413F
:10F9F0004FF6FF734A899A42DCD0BDF815E08B8937
:10FA000073449BB28B8109888E4501D19A420CD8F0
:10FA10008AB3B2FBF1F001FB102080B258BB122078
:10FA200000FB0540807B012825D1D21A8A42D8BF2D
:10FA300091B2122202FB0544C9B9D4F80230C9F8C8
:10FA40000430A9F802102DE70A78012ACDD1FF2051
:10FA50000870194603A80193FFF7F4FB019B06F811
:10FA600038301A46194603A8FFF7CAFCBDE7D4F898
:10FA700006201344E3E7122202FB0544D4F80620D3
:10FA8000ADF815304FF0FF330492A372E37291E7A3
:10FA90005680FF1F13460A46194601F08BB900BF76
:10FAA00030B50329039C04981DD12BB9164A226056
:10FAB00004220280002030BD40F209418B420FD168
:10FAC000022A4FF000030CD810490C2505FB031344
:10FAD000D9681B6951F8221021609B5C0380E9E71B
:10FAE00001230122F0E7072901D9CD2030BD074BC2
:10FAF00003EB8102126A2260002AF6D003EB410375
:10FB0000B3F84030EAE700BF5780FF1F64130100DD
:10FB100001299FBF034B5B5C1370002088BFCD2081
:10FB2000704700BF5493FF1F01299DBF024B002067
:10FB30005A54CD20704700BF5493FF1F19B14B1E7C
:10FB400058425841704701207047054B1A788A4245
:10FB500004D05878431A58425841704701207047E2
:10FB60005493FF1F0020704700487047B4130100F2
:10FB700001299FBF044BC1EBC101C918002094BFEC
:10FB80001160CD20704700BF5B80FF1F012930B599
:10FB90000ED8084DC1EBC10108231068C45CC81819
:10FBA000284401330F2B00F8084CF6D1002030BD5B
:10FBB000CD2030BD5B80FF1F01299FBF034B03EBAE
:10FBC00041010020116088BFCD2070475693FF1F70
:10FBD00001299FBF034B03EB41010020116088BF47
:10FBE000CD2070475A93FF1F01290AD8136818784F
:10FBF000054B03EB4101887013685B78CB700020E4
:10FC00007047CD20704700BF5493FF1F01290AD8C9
:10FC100013681878054B03EB4101887113685B7812
:10FC2000CB7100207047CD20704700BF5493FF1F59
:10FC3000084B5A7803F8022BFF210022D1540132DD
:10FC4000072AFBD1044A0023052199540133072BCD
:10FC5000FBD170475E93FF1F6793FF1F00BF704784
:10FC6000013AD2B2062A10B51C4608D8054B5A7084
:10FC7000FFF7DEFF2146BDE81040FFF7C9B9992024
:10FC800010BD00BF5E93FF1F024B00225A70FFF7AA
:10FC900031BA00BF5E93FF1F37B50F4C257805B909
:10FCA000C1B98DF802308DF800109DF81830ADF80C
:10FCB000032069469DF81C2000788DF80130FFF77D
:10FCC00037FA9DF800301BB110B92378013B23703F
:10FCD00003B030BD9520FBE75E93FF1F38B50A4B9C
:10FCE0000D461C7859788C421C4600D14DB92946E6
:10FCF0000078FFF7D1FA2DB120B9237801332370B2
:10FD000038BD962038BD00BF5E93FF1F4B1E062BEB
:10FD100005D8094B19444B78137000207047CB0667
:10FD200007D501F00F01062903D8034B19444B7A7C
:10FD3000F2E78220704700BF5E93FF1F4B1E062B29
:10FD40002DE9F0418046174605D8174B19444A70F3
:10FD50000020BDE8F081CB0622D501F00F05062D6D
:10FD60001ED8012A4FEAD1140F4E06D12246294649
:10FD7000FFF7C6FA35446F72EAE7002AFAD1731921
:10FD80005B7A012BF6D122462946FFF789FB002D2D
:10FD9000F0D184F0010229464046FFF781FBE9E7F4
:10FDA0008220BDE8F08100BF5E93FF1F00207047F6
:10FDB000062903D9A1F11003072B07D8044B53F8E8
:10FDC0002130002B0CBFC42000207047C420704796
:10FDD000DC130100102810B50C4601D1FFF728FFF5
:10FDE000034B53F820300BB120469847002010BD3C
:10FDF000DC1301001FB5144602228DF807001A809B
:10FE000005210DF10F020DF10700FFF77FFF034BF6
:10FE10009DF80F201A80236004B010BD7093FF1F5F
:10FE20001FB5144601228DF807001A8004210DF138
:10FE30000F020DF10700FFF769FF044B9DF80F203B
:10FE40001A800020236004B010BD00BF7093FF1F14
:10FE5000F0B5002685B01E8049888DF80700ADF802
:10FE60000E10FFF76BFE18B3BDF80E20114F04AC57
:10FE7000B2FA82F2520901210DF10700FFF75EFF8D
:10FE800034F8022D0421D2B20DF10700FFF756FF1E
:10FE90007B682246012105469DF8070098477B684C
:10FEA0009DF80700324602219847284605B0F0BD6C
:10FEB0000425FAE77093FF1F73B502AC002504F820
:10FEC000010D0E461D80042201212046FFF736FF5A
:10FED0007288024B28461A7202B070BD7093FF1FE1
:10FEE00013B54C8889888DE80C000B46E2B2210AD4
:10FEF000FFF7D6FD02B010BD2DE9F04186B01746E0
:10FF00001E4606AA00238846059303238DF80F009A
:10FF100002F8083D01210DF10F00FFF7F7FE98F8F8
:10FF20000050274C15F0030528D10DF111020621D0
:10FF30000DF10F00FFF7EAFE9DF811309DF80F005C
:10FF400003F0030323800DF11203019305AB00932B
:10FF50002A462B460221FFF7A3FD059BDB7913F010
:10FF6000400F238814BF43F0010323F001032380D3
:10FF7000022333803C6006B0BDE8F081012D08D13A
:10FF80009DF81030012B02D198F80430ABB9002352
:10FF9000EDE7022DEED198F8041041F010010DF1BB
:10FFA0001202C9B20DF10F00FFF7B0FE9DF812303A
:10FFB00003F0010323803580DCE7CD20DAE700BFC2
:10FFC0007093FF1F7FB500221A800B784E788DF852
:10FFD000070013F003030D46C6F3400634D1FEB10B
:10FFE0004B88013B9BB2012B52D80DF10F02062129
:10FFF0000DF10700FFF78AFE044670B9AB780122C5
:020000021000EC
:100000009A409DF80F301A43D2B206210DF1070035
:100010008DF80F20FFF792FE0446204604B070BD15
:100020004E88012E34D10DF10F0206210DF107008B
:10003000FFF76CFE04460028EFD1AA7896409DF8A1
:100040000F2022EA0602E0E7022B21D109798DF880
:100050000F10324641F010010DF10700FFF76EFE60
:100060006B78002E14BF07210821012B044607D10D
:100070009DF80F00C10900F00F00FFF7ADF908214E
:10008000044B9DF807005B680DF10F029847C4E729
:10009000CD24C2E77093FF1F10B500241C800B789D
:1000A00003F00303012B05D18A780979FFF73CFDA2
:1000B000204610BD042010BD38B515460A7802F060
:1000C0000302012A07D1054C1A8009792246FFF75D
:1000D0001FFD2C6038BD042038BD00BF7093FF1F8A
:1000E00013B5CD298DF8070007D1012290210DF11C
:1000F0000700FFF723FE02B010BD0D491C88088AD7
:100100001268844288BF18800C461B889DF807003F
:100110000021FEF74DFF94F90A30002BEBDA0023A3
:100120001A4619460DF10700FFF76AF9E3E700BF29
:100130007093FF1F73B5054600266A4601218DF8AE
:1001400000600196FFF7E2FDAA78434C012A52D1E4
:1001500068680368C4F80A304368A07AC4F80E30AF
:1001600004F10A0110F0600F1ED1E27A3B4B53F804
:100170002240002C3DD09DF80000022839D802EB27
:1001800042021344034493F83430012B31D10DF172
:10019000020301AA2878A0470DF1020301AA014633
:1001A0002878FFF79DFF13E0238AADF80230202B5B
:1001B00017D87BB102060DD40A68C4F812204A6829
:1001C000C4F81620314604F11A022846FFF718F940
:1001D00002B070BDE46B64B10DF1020301AA2049C5
:1001E000D8E702A82B7800F8073D9021FFF7A6FD7D
:1001F000EEE7CD20D0E79DF80030042B10D12B780E
:10020000217A02AD05F8063D2846FFF7D1F9012213
:1002100011462846FFF792FD227A03212846E5E79A
:1002200094F90A30002BD3DBEB78002BD0D1E66BAE
:1002300086B1B5F8093028780833ADF8023004F1FA
:1002400012010DF1020301AAB04701460DF10203AC
:1002500001AAA5E7CD21F9E77093FF1F3C14010027
:100260007A93FF1F034B5960DA630021024AFFF7BC
:100270009DBD00BF7093FF1F3501010007B502ABA4
:10028000054A03F8010D002118465160D163FFF7BC
:100290008FFD03B05DF804FB7093FF1F00207047D3
:1002A000354B41F248015A5822F00F0242F0020247
:1002B0005A5041F204015A5842F480225A5041F2F5
:1002C00034015A5842F480225A5003F52C336021ED
:1002D00093F8942042F0020283F89420C02283F81D
:1002E0000021FF221A7483F8802083F8882083F885
:1002F0008420002283F88C2083F80C111F491A7582
:10030000080A00F0FE0083F8982083F8C02083F8E4
:10031000C42083F8C82083F8CC2083F8D02083F849
:10032000D42083F8D82083F8DC2083F8E02083F8F9
:10033000E42083F8E82083F8EC2083F8F02083F8A9
:10034000F42083F8F82083F8FC2083F89C00C1F3A4
:100350000740090E83F8B00083F8B41083F8AC208E
:100360001A7783F8082193F8942002F0D40242F01F
:10037000010283F89420704700700440009EFF1F24
:10038000024B4FF400125A60704700BF00E100E0DA
:10039000034B4FF40012C3F884215A60704700BF2A
:1003A00000E100E008B5FEF782F910B9FFF7F0FFB1
:1003B00008BD1B2008BD00BF034B4AF202629A81B0
:1003C0004BF280429A8170470020054081F0004145
:1003D00002E000BF83F0004330B54FEA41044FEA2A
:1003E000430594EA050F08BF90EA020F1FBF54EAC5
:1003F000000C55EA020C7FEA645C7FEA655C00F061
:10040000E2804FEA5454D4EB5555B8BF6D420CDD31
:100410002C4480EA020281EA030382EA000083EAB4
:10042000010180EA020281EA0303362D88BF30BD54
:1004300011F0004F4FEA01314FF4801C4CEA1131AA
:1004400002D0404261EB410113F0004F4FEA033309
:100450004CEA133302D0524263EB430394EA050F94
:1004600000F0A780A4F10104D5F1200E0DDB02FA03
:100470000EFC22FA05F2801841F1000103FA0EF297
:10048000801843FA05F359410EE0A5F120050EF15D
:10049000200E012A03FA0EFC28BF4CF0020C43FA8E
:1004A00005F3C01851EBE37101F0004507D54FF09B
:1004B000000EDCF1000C7EEB00006EEB0101B1F5EB
:1004C000801F1BD3B1F5001F0CD349085FEA300031
:1004D0004FEA3C0C04F101044FEA445212F5800F3C
:1004E00080F09A80BCF1004F08BF5FEA500C50F1D9
:1004F000000041EB045141EA050130BD5FEA4C0CBC
:10050000404141EB010111F4801FA4F10104E9D144
:1005100091F0000F04BF01460020B1FA81F308BF3B
:100520002033A3F10B03B3F120020CDA0C3208DD07
:1005300002F1140CC2F10C0201FA0CF021FA02F1E2
:100540000CE002F11402D8BFC2F1200C01FA02F152
:1005500020FA0CFCDCBF41EA0C019040E41AA2BF77
:1005600001EB0451294330BD6FEA04041F3C1CDA3F
:100570000C340EDC04F11404C4F1200220FA04F05F
:1005800001FA02F340EA030021FA04F345EA030109
:1005900030BDC4F10C04C4F1200220FA02F001FACB
:1005A00004F340EA0300294630BD21FA04F029464D
:1005B00030BD94F0000F83F4801306BF81F48011E6
:1005C0000134013D4EE77FEA645C18BF7FEA655C59
:1005D00029D094EA050F08BF90EA020F05D054EA2B
:1005E000000C04BF1946104630BD91EA030F1EBF30
:1005F0000021002030BD5FEA545C05D14000494134
:1006000028BF41F0004130BD14F580043CBF01F526
:10061000801130BD01F0004545F0FE4141F470010C
:100620004FF0000030BD7FEA645C1ABF19461046E7
:100630007FEA655C1CBF0B46024650EA013406BFE8
:1006400052EA033591EA030F41F4002130BD00BFA7
:1006500090F0000F04BF0021704730B54FF4806464
:1006600004F132044FF000054FF0000150E700BFE5
:1006700090F0000F04BF0021704730B54FF4806444
:1006800004F1320410F0004548BF40424FF0000131
:100690003EE700BF42004FEAE2014FEA31014FEA74
:1006A00002701FBF12F07F4393F07F4F81F06051C3
:1006B000704792F0000F14BF93F07F4F704730B532
:1006C0004FF4607401F0004521F0004120E700BFC5
:1006D00050EA010208BF704730B54FF000050AE04C
:1006E00050EA010208BF704730B511F0004502D54D
:1006F000404261EB41014FF4806404F132045FEA4F
:10070000915C3FF4DCAE4FF003025FEADC0C18BFF3
:1007100003325FEADC0C18BF033202EBDC02C2F1E9
:10072000200300FA03FC20FA02F001FA03FE40EA7B
:100730000E0021FA02F11444C1E600BF70B54FF07B
:10074000FF0C4CF4E06C1CEA11541DBF1CEA13555D
:1007500094EA0C0F95EA0C0F00F0DEF82C4481EAC5
:10076000030621EA4C5123EA4C5350EA013518BFE5
:1007700052EA033541F4801143F4801338D0A0FBD2
:1007800002CE4FF00005E1FB02E506F00042E0FB7F
:1007900003E54FF00006E1FB03569CF0000F18BF85
:1007A0004EF0010EA4F1FF04B6F5007F64F540742D
:1007B00004D25FEA4E0E6D4146EB060642EAC621C0
:1007C00041EA55514FEAC52040EA5E504FEACE2E2D
:1007D000B4F1FD0C88BFBCF5E06F1ED8BEF1004F30
:1007E00008BF5FEA500E50F1000041EB045170BDAC
:1007F00006F0004646EA010140EA020081EA0301F0
:10080000B4EB5C04C2BFD4EB0C0541EA045170BDEB
:1008100041F480114FF0000E013C00F3AB8014F165
:10082000360FDEBF002001F0004170BDC4F10004AE
:10083000203C35DA0C341BDC04F11404C4F120052F
:1008400000FA05F320FA04F001FA05F240EA02008A
:1008500001F0004221F0004110EBD37021FA04F6C0
:1008600042EB06015EEA430E08BF20EAD37070BD7A
:10087000C4F10C04C4F1200500FA04F320FA05F0D9
:1008800001FA04F240EA020001F0004110EBD370DB
:1008900041F100015EEA430E08BF20EAD37070BD4B
:1008A000C4F1200500FA05F24EEA020E20FA04F324
:1008B00001FA05F243EA020321FA04F001F00041D3
:1008C00021FA04F220EA020000EBD3705EEA430E44
:1008D00008BF20EAD37070BD94F0000F0FD101F073
:1008E0000046400041EB010111F4801F08BF013CAC
:1008F000F7D041EA060195F0000F18BF704703F0EA
:100900000046520043EB030313F4801F08BF013D70
:10091000F7D043EA0603704794EA0C0F0CEA13552C
:1009200018BF95EA0C0F0CD050EA410618BF52EAE6
:100930004306D1D181EA030101F000414FF00000EC
:1009400070BD50EA410606BF1046194652EA4306FA
:1009500019D094EA0C0F02D150EA013613D195EA6E
:100960000C0F05D152EA03361CBF104619460AD1B6
:1009700081EA030101F0004141F0FE4141F47001C0
:100980004FF0000070BD41F0FE4141F4780170BDB0
:1009900070B54FF0FF0C4CF4E06C1CEA11541DBF15
:1009A0001CEA135594EA0C0F95EA0C0F00F0A7F817
:1009B000A4EB050481EA030E52EA03354FEA013144
:1009C00000F088804FEA03334FF0805545EA131357
:1009D00043EA12634FEA022245EA111545EA10651F
:1009E0004FEA00260EF000419D4208BF964244F1B6
:1009F000FD0404F5407402D25B084FEA3202B61AD5
:100A000065EB03055B084FEA32024FF480104FF4A8
:100A1000002CB6EB020E75EB030E22BFB61A75461C
:100A200040EA0C005B084FEA3202B6EB020E75EBAF
:100A3000030E22BFB61A754640EA5C005B084FEA17
:100A40003202B6EB020E75EB030E22BFB61A7546E4
:100A500040EA9C005B084FEA3202B6EB020E75EBEF
:100A6000030E22BFB61A754640EADC0055EA060EB0
:100A700018D04FEA051545EA16754FEA06164FEAF3
:100A8000C30343EA52734FEAC2025FEA1C1CC0D19F
:100A900011F4801F0BD141EA00014FF000004FF02C
:100AA000004CB6E711F4801F04BF01430020B4F1ED
:100AB000FD0C88BFBCF5E06F3FF6AFAEB5EB030CA5
:100AC00004BFB6EB020C5FEA500C50F1000041EBA2
:100AD000045170BD0EF0004E4EEA113114EB5C046F
:100AE000C2BFD4EB0C0541EA045170BD41F4801142
:100AF0004FF0000E013C90E645EA060E8DE60CEA4A
:100B0000135594EA0C0F08BF95EA0C0F3FF43BAF66
:100B100094EA0C0F0AD150EA01347FF434AF95EA1D
:100B20000C0F7FF425AF104619462CE795EA0C0F01
:100B300006D152EA03353FF4FDAE1046194622E7CE
:100B400050EA410618BF52EA43067FF4C5AE50EAA8
:100B500041047FF40DAF52EA43057FF4EBAE12E798
:100B60004FF0FF3C06E000BF4FF0010C02E000BF79
:100B70004FF0010C4DF804CD4FEA410C7FEA6C5C5C
:100B80004FEA430C18BF7FEA6C5C1BD001B050EAFF
:100B9000410C0CBF52EA430C91EA030F02BF90EAEA
:100BA000020F0020704710F1000F91EA030F58BFA9
:100BB000994208BF90422CBFD8176FEAE37040F00B
:100BC000010070474FEA410C7FEA6C5C02D150EAA9
:100BD000013C07D14FEA430C7FEA6C5CD6D152EA64
:100BE000033CD3D05DF8040B704700BF8446104629
:100BF00062468C461946634600E000BF01B5FFF728
:100C0000B7FF002848BF10F1000F01BD4DF808EDF7
:100C1000FFF7F4FF0CBF012000205DF808FB00BFC8
:100C20004DF808EDFFF7EAFF34BF012000205DF822
:100C300008FB00BF4DF808EDFFF7E0FF94BF01206F
:100C400000205DF808FB00BF4DF808EDFFF7CEFF70
:100C500094BF012000205DF808FB00BF4DF808EDAF
:100C6000FFF7C4FF34BF012000205DF808FB00BF80
:100C70004FEA410212F5001215D211D56FF47873C4
:100C8000B3EB625212D94FEAC12343F0004343EA67
:100C9000505311F0004F23FA02F018BF4042704742
:100CA0004FF00000704750EA013005D111F00040CC
:100CB00008BF6FF0004070474FF00000704700BF62
:100CC000FDF7BDFB002103E00A4B5B5843500431A4
:100CD00009480A4B42189A42F6D3094A02E0002317
:100CE00013600432074B9A42F9D300F00DF88047A5
:100CF00070470000C81401000880FF1F6C85FF1FAB
:100D00000086FF1F24A2FF1F274C08B5F7F7B9FB89
:100D1000F7F720FCF7F786FDF7F798FDF7F7A2FC49
:100D2000F7F764FFFCF78EFBFCF776F9F8F7CAF8E3
:100D3000F7F728FEE08CF7F71BFF2078F7F7A2FC07
:100D4000E078F7F70FFDF7F7C6FE28B1F7F7C3FE17
:100D50006070F7F7C0FEA060F7F724FF2189607983
:100D6000228AFCF7B3F9FDF7E3F8FDF781FA0F4BA0
:100D70004FF400725A60FAF78BFEFBF76BFB0C4BDB
:100D800004225A60FAF7B6FFFBF788FBFBF763FB18
:100D9000F7F7A8FEF7F7DCFE0028F3D0FDF7C8F858
:100DA000FAF776FEEEE700BF0C80FF1F80F00F40E1
:100DB00000F00F4070B4860746D0541E002A41D080
:100DC000CAB2034602E014F1FF343BD303F8012B0F
:100DD0009D07F8D1032C2ED9CDB245EA05250F2C5D
:100DE00045EA054519D903F110022646103E0F2E9B
:100DF00042F8105C42F80C5C42F8085C42F8045C73
:100E000002F11002F2D8A4F1100222F00F0204F055
:100E10000F041032032C13440DD91E462246043A07
:100E2000032A46F8045BFAD8221F22F00302043298
:100E3000134404F003042CB1C9B21C4403F8011B91
:100E40009C42FBD170BC704714460346C2E700BF0A
:100E50002DE9F84355EC104BC5F30A52A2F2FF33CB
:100E6000132B064612DC002B41DB244A42FA03F323
:100E700005EA030252EA040017D105F000430246D6
:100E800086ED000B43EC102BBDE8F883332B1CDC04
:100E9000A2F213424FF0FF3323FA02F214EA0207E0
:100EA0001CD0A94624EA020803E04FF0000825EA16
:100EB000030942464B4620462946C6E90023FFF770
:100EC00089FA41EC100BBDE8F883002205F00043DD
:100ED00086ED000B43EC102BBDE8F88305F00043D2
:100EE0003A4686ED000B43EC102BBDE8F883002258
:100EF00005F00043C6E90023BDE8F883FFFF0F00BB
:100F0000024B13B1024800F005B870470000000022
:100F1000210F0100002301461A46184600F01EB8B2
:100F200038B50A4C0A4D641BA4100AD004F1804362
:100F3000013B05EB8305013C55F804399847002C2B
:100F4000F9D1BDE8384000F0B3BA00BFC8140100C1
:100F5000C4140100704700BF704700BF2DE9F8437B
:100F60002C4D0646286898460F469146FFF7F2FF3B
:100F7000294B1C68D4F84831002B3ED05A681F2AF0
:100F80001CDC02F1010E76B103EB82010124C1F8F1
:100F90008890D3F8880194402043022EC3F888013A
:100FA000C1F8088123D00232C3F804E0286843F86E
:100FB0002270FFF7D1FF0020BDE8F883174B0BB379
:100FC0004FF4C870AFF300800346D8B1D4F848217D
:100FD0000260002141600A46C4F848014FF0010E4A
:100FE000C0F88811C0F88C11002EDCD0CCE7D3F803
:100FF0008C110C43C3F88C41D5E704F5A673C4F8F3
:101000004831BBE72868FFF7A7FF4FF0FF30BDE886
:10101000F88300BF6885FF1FA014010000000000D6
:1010200051EC100B2DE9F843C1F30A59A9F2FF3531
:10103000132D0C4610EE106A884610EE107A22DC52
:10104000002D52DB3E4B43FA05F901EA0903034345
:101050001ED039A3D3E90023FFF7BEF900220023F5
:10106000FFF7FCFD48B1002C04DD4FF4801343FA78
:1010700005F5A84428EA0904002723463A4643EC2C
:10108000102BBDE8F883332D06DDB5F5806F3FD01A
:1010900041EC100BBDE8F883A9F213494FF0FF3380
:1010A00023FA09F910EA090FF2D023A3D3E90023A8
:1010B000FFF792F900220023FFF7D0FD0028DCD0D3
:1010C000002C09DD142D32D00127C5F1340507FAB3
:1010D00005F5AE1928BFB844444626EA0907234659
:1010E0003A4643EC102BBDE8F88313A3D3E9002361
:1010F000FFF772F900220023FFF7B0FD0028BCD0F3
:10110000002C10DB54EA06070BD000270D4CB4E787
:1011100010EE102A0B46FFF75FF941EC100BBDE80B
:10112000F8833C46A9E700274FF00044A5E704F107
:101130000108D1E7AFF300809C7500883CE4377E5E
:10114000FFFF0F000000F03F51EC100BC1F30A53FA
:101150002DE9F041A3F2FF35132D0C460F4610EE9A
:10116000106A1DDC002D43DB3D4B43FA05F801EA14
:101170000803034319D038A3D3E90023FFF72CF960
:1011800000220023FFF76AFD20B1002C49DB27EA8B
:10119000080400262346324643EC102BBDE8F081BC
:1011A000332D06DDB5F5806F32D041EC100BBDE874
:1011B000F081A3F213434FF0FF3828FA03F810EA46
:1011C000080FF2D024A3D3E90023FFF705F900228A
:1011D0000023FFF743FD0028DCD0002C27DB3C4632
:1011E00026EA08062346324643EC102BBDE8F08180
:1011F00019A3D3E90023FFF7EFF800220023FFF73C
:101200002DFD0028C6D0002C1CDB00263446C1E78B
:1012100010EE102A0B46FFF7DFF841EC100BBDE88B
:10122000F0814FF4801343FA05F52F44AFE7142DF6
:1012300010D00123C5F1340503FA05F5AE1928BF16
:10124000FF18CCE724F00042064B324318BF1C467F
:1012500000269FE70137C2E79C7500883CE4377E93
:10126000FFFF0F000000F0BF8025000040380000A5
:10127000004B0000807000000096000000E10000BC
:10128000002C010000C201000084030090D0030084
:1012900020A1070040420F0050C300008813000047
:1012A000018008080000000000000000C8000000E5
:1012B0000100C800008000000000000000000000E5
:1012C000000000000000000000000000000000001E
:1012D00000000000000000000100020004000800FF
:1012E00010002000010101000100000000000000CA
:1012F00000000000000100000000000000010000EC
:1013000000000000010101000000000000000000DA
:1013100000010000000000000101010001010001C6
:1013200001000000010101000000000000000000B9
:1013300000010000000000000101010001010001A6
:10134000010000000000000000000000000001019A
:101350000100000100000000000000000000010189
:10136000010000015780FF1F040000000904000075
:10137000C8130100D81301000000000000000000A5
:1013800000000000000000002E81FF1FEB80FF1F07
:10139000000000000000000000000000000000004D
:1013A00000000000000012004300000000000000E8
:1013B00000000000030102011000020200100003FF
:1013C00003011000000100005780FF1FB180FF1FC4
:1013D0008B80FF1F6980FF1F043A26223501010020
:1013E00031EA0000C9EA000039E800005DFC0000B5
:1013F0005DFC00005DFC00005DFC00005DFC000089
:101400005DFC00005DFC00005DFC00005DFC000078
:101410005DFC00005DFC00005DFC0000BBED000019
:1014200051ED0000B1ED00007DED000051ED000038
:101430005DFC00003DED000029EE0000F9FE00001B
:10144000C5FF000000000000C5FF00000000000014
:10145000B9FE0000E1FE00000000000021FE0000D7
:1014600051FE0000B900010099000100F5FD0000E7
:101470000101000101000000000101000000000066
:101480000101010101000000010100010100010052
:101490000001000001000036323130563130370093
:1014A0004081FF1FF8B500BFF8BC08BC9E467047DE
:0C14B000F8B500BFF8BC08BC9E467047B1
:0814BC00010F0100358400005E
:0414C400118400008F
:1014C800971401000001020000080000010000005C
:1014D8000200000000000000000000000000000002
:1014E80000000000000000000000000000000000F4
:1014F80000000000000000000000000000000000E4
:1015080000000000A1200000000002000000FF040D
:1015180003090400C20100000008000000000000E8
:1015280000220342004100440020005300540052AE
:101538000049004E004700200049004E0044004585
:1015480000580026035300740065007000700065A1
:1015580000720020004D006F0074006F00720020C0
:101568000044006500760020003A03540052004908
:10157800004E0041004D004900430020004D006F1F
:1015880000740069006F006E00200043006F006E59
:1015980000740072006F006C002000200020002002
:1015A80000200009024300020100C03209040000C3
:1015B80001020200000524001001052401010104B4
:1015C80024020605240600010705830310000A0902
:1015D800040100020A00000007058102100000074C
:1015E80005020210000012010002020000103C2A4D
:1015F8000001020001020001000000002C84FF1F0E
:101608009484FF1FFC84FF1F0000000000000000FE
:1016180000000000000000000000000000000000C2
:1016280000000000000000000000000000000000B2
:1016380000000000000000000000000000000000A2
:101648000000000000000000000000000000000092
:101658000000000000000000000000000000000082
:101668000000000000000000000000000000000072
:101678000000000000000000000000000000000062
:101688000000000000000000000000000000000052
:101698000000000000000000000000000000000042
:1016A80001000000000000000E33CDAB34126DE6DF
:1016B800ECDE05000B000000000000000000000048
:1016C8000000000000000000000000000000000012
:1016D8000000000000000000000000000000000002
:1016E80000000000000000000000000000000000F2
:1016F80000000000000000000000000000000000E2
:041A280000A2FF1FFA
:101A2C00C81401000880FF1F6405000000000000BE
:081A3C000000000000000000A2
:020000020000FC
:020000041FFFDC
:04800000000000007C
:0400000310000CC11C
:00000001FF
